:020000041100E9
:10300000F7B5164B0192C318021D002000938823C8
:103010005B05D3181B685C1C1AD09CB2402C18D8D6
:103020008D781E0CAC466746CD782D023D43AE42EE
:1030300006D1019800280ED110000C70240A4C70A3
:1030400003249BB20733A343D218009B9A42DED3DA
:10305000FEBD4432F9E71000FAE7C046FC0F00005D
:10306000802213B503000324019189B25201073174
:103070009B18A14304305A1A88235B05C3181B68A8
:10308000591C03D190429241104016BD99B240297B
:1030900007D80B000733A343C0189042ECD300209D
:1030A000F3E74430F9E7134B134A1B68126810B575
:1030B000F424934201D81A00F024104BA4021B6898
:1030C0009A4210D813000E4A12689A420ED3013366
:1030D00007D1F0239B029C4203D10A49054808F01E
:1030E0006BFA200010BDF824A402ECE7FC24A40233
:1030F000F7E7C04600C0031100D0031100E0031140
:1031000000F00311FFFFFF7FF0B59BB015000490A6
:103110000391402A00D9A0E006AB59801A80FFF73E
:10312000C2FF0400042816D9002206A9FFF768FF91
:10313000052810D906AB1B88AB420CD1002D07D057
:10314000514B2A000499C01808F026FA002802D131
:1031500001201BB0F0BD06AB1D8020000699FFF7D3
:103160007FFF041E7BD1069B0793FFF79CFF802304
:103170005B01C61880230700DB029E4201D3F026C4
:10318000B60288235B05F31801931B68013302D054
:10319000019807F0F1FF3D49019808F00DFA3B1D39
:1031A0000293331D05938822029B52059B181B68CE
:1031B00008935A1C3CD044219AB20091402A04D86A
:1031C0000320D11D814389B2009103991B0C8B42CE
:1031D00024D0402A22D80122300008A9FFF710FF8E
:1031E000021E1BD1380008A9FFF70AFF04000428BB
:1031F00031D9009A059B9B1880225201B218934244
:1032000040D288235B05C118009A09A807F0A4FFE3
:103210001D4B009A09A9F01808F0F6F8009A029BD5
:103220009446634402931A4B029AFB189A42BAD30B
:1032300088235B05FC1821680198013908F0BCF966
:10324000200007F099FF039A07AB5A8030000799D6
:10325000FFF706FF0400002C03D1002079E70428C3
:10326000FBD988235B05E018069908F0A5F903232C
:10327000EA1C9A4300D16BE7034B0499E01808F06D
:10328000C3F865E70424ECE704000011FFFFFF7FAB
:10329000F80F0000F7B505001400402A21D80027D8
:1032A00001AE71803780FFF7FEFE042816D93A0080
:1032B0003100FFF7A5FE042810D93688BC420BD098
:1032C000BD4209D0221CB44200D9321C064B92B236
:1032D000C118280007F040FF30B2FEBDC04300B265
:1032E000FBE703204042F8E70400001137B5042251
:1032F00004000D0001A81649FFF7CCFF02000428C6
:103300000BD1019BA34208D3AB4204D0104901A8C2
:103310000195FFF7F9FE01203EBD0E4C2368200009
:10332000019307F029FF019920000139019108F06C
:1033300043F980235B01E418074B9C42EED1042241
:10334000034901A80195FFF7DFFE0020E4E7C0462E
:103350005555000000C003110000041130B589B0BC
:1033600007F0E2FE10226946254808F015F8254BC3
:10337000009A9A420ED1019B029A0F2B33D800215A
:1033800001240698013B08D2002900D00292029B3A
:10339000013331D10023029325E0551CF2D1020004
:1033A0002100EFE710341022200004A907F0F4FFF9
:1033B000029B013301D1069B0293882304995B058C
:1033C000C918059B06981A03120B049105928142B5
:1033D00003D02B4201D107F0BFFE019B013B0193BB
:1033E000019B002BDED1029B002B03D00493049899
:1033F0004168084709B030BDE025014C2D03EFE7D7
:1034000000000111504859368022F8B5964C974B70
:10341000D200002120001C6008F0EEF82300944A3E
:1034200088331A60934B1A786A23002A00D011332C
:10343000E3620A232365904B37221B780820A3639D
:103440008E4B2118E361102323628D4B3B25636172
:10345000C823DB00A36123008C331A602823013AC0
:10346000E26320646364CA67043A211DCA672100CD
:10347000BC310D602100C03108602100C4310B60F7
:1034800021000635CC310D602100083DC8310D60AA
:103490002100D0310A602200D43210602200D832DC
:1034A000136022000227E032210017604222DC3143
:1034B0000A6021001B3DE4310D602100E831086005
:1034C0002100EC310B6023000521F4331960230047
:1034D000F0331A602300183290331A6023009433BB
:1034E000186023001E3A98331A60AF23DB00236074
:1034F000644BFA262363644B644DE360644BF03104
:10350000A3642300FF31FC33B600A16021611E607B
:10351000A5627325E5656D3D6565A56596255D4AE2
:10352000AD00E264666258606766A56600270925FB
:10353000A767E566584F594D606720002567E26729
:103540003A6015279C30676007001A203860200019
:10355000A0300700212038602000A83007004C4828
:1035600038602000F830066026006427A4363760F3
:1035700026005F3FAC3637602600033FB036376029
:103580002600C637B436376026000027B8363760C5
:1035900038269E60424E96205E64424E5A66DE6138
:1035A000414E9A645E62F53EFF3E9E621E269A6719
:1035B000354A8000DE661F675F67DD651D6618623D
:1035C000DA67BE23394A5B00E250394BD8382350C2
:1035D00004302250C4225200A350C623E4205B00D2
:1035E000E1500433334AE1503349344BD16034491C
:1035F000800019503349E938FF38195032490430F6
:10360000195032493248D16132491163324951630C
:103610001900F4310860CE20304940001160304973
:10362000195019002F48F83108602F49D1658221BF
:103630002E4A89005A501A002D490832D1671A00C3
:103640002C49B432116088212B4A89005A501A0043
:103650002A49883211602A4ADA6407F0C5FD012040
:1036600008F04AF8F8BDC0460004FF1F8064FF1F41
:10367000506FFF1F2044FF1F4A0AFF1F3A07000038
:1036800080C3C9019A020000DC0500006A1800002E
:1036900050C3000088130000F009FF1F204E0000F7
:1036A0006509FF1F68100000C409000040420F00B8
:1036B00010270000FC00FF1F751CFF1F0000FF1FEC
:1036C000C92CFF1F5130FF1FE92EFF1F3520FF1FA0
:1036D0002527FF1F5120FF1FFD21FF1FC11FFF1FB7
:1036E0004929FF1F312AFF1F8D19FF1F5528FF1F72
:1036F0007925FF1F8525FF1FC11EFF1F791FFF1F93
:10370000391EFF1F0223F0B50124634D634E2B7059
:10371000634B8BB01C70634F039333680021092007
:10372000BB7006F021FC092006F028FB031E05D122
:10373000BA78552A02D0332A00D0A0E000233360A3
:10374000042006F06FFD07F067FEFFF75DFE07F04F
:103750001BFE1F2201240021534B1E261A70534BBF
:103760001C70534B1970534B19689143163A0A4316
:103770001A60602219689143403A0A431A6007F0C0
:10378000ABFD07F029FD4C4B9847C120FF214B4B67
:1037900080001A588A431A50C522920098588843CC
:1037A000BF39014399509858454908408021C901C3
:1037B0000143802099509958C0050902090A014324
:1037C000995080213F48490107F09EFD03232200C4
:1037D00000933D4901943D4807F0CEFE16223C4936
:1037E00004A807F0B9FC02AB04ACF61861782078A5
:1037F000023406F0D3FAA642F8D1364C0320012158
:1038000006F0E0FB2268344B03201A40A023DB02C1
:1038100013432360802322689B04134323602268A0
:103820002E4B1A4080239B03134323602C4A2D4BBD
:10383000934200D8012007F097FD07F035FE802362
:103840002268DB0413432360287807F0D5FC039B30
:103850001878C0B207F018FF07F04EFD2249042087
:1038600007F05AFD06F0AAFC00F040F800F08EFDCB
:1038700000F036FE00F0B8FB00200BB0F0BD009069
:103880002100194A042007F067FD8023DB059C62B4
:10389000FFF764FD54E7C0464A0AFF1F34F00040BA
:1038A0002044FF1F2862FF1F480AFF1F490AFF1F0D
:1038B000680AFF1FBCF00040E1A2000000E100E048
:1038C000FF00FFFF2444FF1FA856FF1F2454FF1FC3
:1038D00098B7001114F00040FF7FF8FFFFFF9FFF33
:1038E0000080FF1F506FFF1F3B000108002210B532
:1038F0001100112007F0B8FE10BD0000F8B500233C
:103900000926374F374C3B62E3681120B343E3602D
:1039100007F02AFF112007F0D7FE112007F02CFF37
:103920004023226880251343236080236268DB02E2
:1039300013436360A3682C4A2B43A360A36802214E
:103940001340A3608023A2689B0113431022A3604D
:10395000236C072093432364236C0F3A134323649F
:1039600080235B003B62226B204B1A402263626B18
:103970001A406263A26B1A40A263E26B1340E363D6
:10398000E3681B4A1340E36006F008FA01210720B0
:1039900006F018FB174B11205A6C15435D6407F0B5
:1039A000E3FBFD21144B154A89005A508023C720A0
:1039B000626B5B0313436363E36880003343E3603C
:1039C0000F4B104A19581140802212020A431A5014
:1039D000802292051A6008220B4B5A63F8BDC0463C
:1039E00000F000403CF00040FFFFDFFFEFFFEFFF83
:1039F000FFFF7FFF003800400000FF1F5118FF1F2E
:103A000000E100E0FF00FFFF0000054007B50422D1
:103A1000044901A807F0A0FB012101A807F0C4FD9B
:103A200007BDC046AEB7001170B52B4C238C002BE0
:103A30002AD0FA22D200934201D2FFF7E7FF228A6E
:103A4000238C002A21D1DA0023826382A382E382BD
:103A500023836383A383E38322606260A260E260C6
:103A60001E4D1F4A6420EB8093420AD8FA220020A0
:103A7000D200934205D91B4A0A21981807F04CFD41
:103A8000C0B200232872238470BD0720E11CCA7FC6
:103A900001320240CA7705D10325201DC17F0131C3
:103AA0002940C17708325200A352002321001A0096
:103AB000088A01321B180231082AF9D1221DD27F4F
:103AC0009200A350626823689B18A2689B18E26862
:103AD0009B185B099BB2C3E72061FF1F0862FF1FB1
:103AE000B70B000030F8FFFF30B503A804880B20A7
:103AF000002C0ED14968074D087849780902014326
:103B00000A20A94205D1012120001980024B1B7A0D
:103B1000137030BD192A00000862FF1FF7B51500A9
:103B200008AA16884A680F4F147852781202224366
:103B30000A24BA4214D10122DBB2019200962A0073
:103B400007F08CFA041E0BD1074B1B68002B07D023
:103B500068782A7800021043424250410130984769
:103B60002000FEBD022900004C61FF1F30B5012579
:103B700003790400BFB02B4211D00A49408806F0F7
:103B8000D9FD28420BD0084B01A95B8D4D800B80DD
:103B9000064B00221B7A60880B7103F0D7FE3FB002
:103BA00030BDC0464461FF1FE040FF1F0862FF1F99
:103BB00010B50549054806F073FD0421044A05487F
:103BC00006F030FD10BDC0464461FF1FFFFF00003E
:103BD000B4B70011E040FF1F10B5024804F038FDF3
:103BE00010BDC0466D3B0011F0B593B005921D00AD
:103BF000DAB20F239B1ADFB20E239B1ADBB20493B7
:103C00001C9B049A023B5B08DB00134306AA13705B
:103C1000199E06AB2A0003900191581C059907F0E4
:103C20009BFA3400002206AB013BBA4252D1002C71
:103C300000D0B9E0102221000AA807F0DDFC0AAB91
:103C4000029306A91A78615C01344A401A70013364
:103C5000102CF6D10AAA1100019807F0BDFB202212
:103C6000212006AB9B18049A05991A7006AB2A000E
:103C7000C01807F071FA01350EAB58193A0000214F
:103C800007F0BAFC2F210123250006AA5218137051
:103C9000002E24D112AB3A003100D81B07F0ACFC47
:103CA000019806AA0EA907F097FB029B06AA925D4F
:103CB0001B7801365340029A1370130001330293AC
:103CC000102EF2D11C9A1B980AA907F045FA002081
:103CD00013B0F0BD01321C74D2B2240AA4E7340040
:103CE000102E00D92C00039B002B19D119002A009B
:103CF00006A807F081FC2200189906A807F02CFA04
:103D0000039B0AAA06A81178185C01334140117080
:103D10000132102BF6D10AAA1100019807F05CFBC2
:103D2000019806AA0EA907F057FB0023189A06A9C6
:103D3000C95CD25C4A401A99CA5401339C42F5D1FD
:103D4000039B012B19D11022002106A807F054FC77
:103D500022001A9906A807F0FFF900230AAA06A86C
:103D60001178185C0133414011700132102BF6D1EB
:103D70000AAA1100019807F02FFB00221A9B361B9C
:103D80001B191A93189B0EA91B191893BA4200D13C
:103D90007EE7CB7B01390133DBB20B74002B00D003
:103DA00076E70132D2B2F1E70120404290E700000D
:103DB00010B5134A134B5179134C19701179200027
:103DC0005970D17899709178D970517812781971A9
:103DD0005A712E2252429A712A32DA7145321A727F
:103DE0000A49313AFFF756FA102808D0102120006E
:103DF00007F0AAF9102220000449FFF785F910BD49
:103E00006509FF1F6061FF1F5061FF1F0DBC0000AF
:103E1000F0B5431805000020114F124A3E8889B0C2
:103E20000C00114956720792320A4A70320ECA705B
:103E300088701E70042639889870090A5970D870E5
:103E40009B19039301940D230849079A0496029540
:103E50000095FFF7C9FE0834E0B209B0F0BDC046D6
:103E60000862FF1F6061FF1F6961FF1F5061FF1F34
:103E7000012202700C4A0300117A41700C209870E4
:103E80009179D970D17919713A21597192789A71D1
:103E90003E22DA71054A117B1972517B5972917B6E
:103EA000D27B9972DA7270470862FF1F1462FF1F9B
:103EB00070B51F4A1F4BD17C04001B681E4A0029A5
:103EC00006D1190604D50323137000F039F870BD2C
:103ED00000211170022219002270013A627005322D
:103EE000A27010322271443A62712A32A2712432D5
:103EF0001140134210D0250041230835E3712800FA
:103F0000FFF7B6FF01002800FFF782FF0430C0B2C0
:103F1000E0700430C0B2DAE740232000E371074BC1
:103F200021721B880A306372FFF7A2FF0630EEE7AA
:103F30001462FF1F2C62FF1F2664FF1F0862FF1F11
:103F400010B5040006220E4907F006F916220D49A5
:103F5000E01D07F001F90C4B1B789B0963770B4BB5
:103F60001A7A0023502A06D840333C2A03D840331B
:103F7000192A00D84033A37100231F20A37710BD56
:103F8000CCB700118F61FF1F8961FF1F0862FF1FFF
:103F900010B5142007F0E0FA124B1422002118602B
:103FA00007F02AFB002007F0FFF8012007F044F992
:103FB000022007F0B1FB032003F0EEFD042005F022
:103FC00003FE052003F02CF8062003F0F9FC07207F
:103FD00001F03EF9082006F005FB092000F0ACFED8
:103FE00010BDC046A861FF1F07F076FA012007F058
:103FF0001BFA07F051F90000094B10B50400984274
:1040000005D0012904D12000064906F049FB10BD66
:104010000229FCD1013904F0D9FA0028F3D0F6E7DF
:10402000FEFF0000CE61FF1F70B50D7A100004AADC
:104030002C00168810221440154220D1002E20D1C9
:104040000A78022A18D14A68517815780E4A09026E
:104050002943914205D00D4A914209D01C800A247F
:1040600004E014220A491A8007F076F8200070BD97
:104070000C2208491A80F7E71C800124F6E708247F
:10408000F4E70B24F2E7C046F3FF0000F4FF000062
:10409000AC42FF1F70B8001110B504000749084872
:1040A00006F0FEFA074804F013FA0020E40704D5EE
:1040B0000721054A054806F0B5FA10BDCE61FF1F7D
:1040C000FFFF0000F93F0011FCB700112441FF1F62
:1040D00000B50C4BBFB01A780B4902A800F0B0FA3B
:1040E0006B4680B2D880002809D06A46074B01A9E8
:1040F0001B889380064B0022188803F027FC3FB0F2
:1041000000BDC046AC61FF1FAD61FF1F7E41FF1FB8
:104110008042FF1F00B50C4BBFB01A780B4902A8B4
:1041200001F05AFB6B4680B2D880002809D06A465D
:10413000074B01A95B8D9380064B0022188803F082
:1041400005FC3FB000BDC046D661FF1FD761FF1F11
:104150002441FF1F8042FF1FF7B50E00377A1C0075
:1041600008AB11003D001A8820231D401F423CD19E
:104170003378022B3BD173681F785B781B023B437B
:104180001E4FBB4208D01E4FBB4214D01D4DAB4248
:1041900021D00A252800FEBD002A2AD1142C2AD8B5
:1041A0002200F06806F0D8FF174B1C70012CF1D9E3
:1041B000FFF7B0FFEEE7002A1BD1202C1BD822000E
:1041C000F06806F0C9FF114B04211C70104B1878E1
:1041D00007F09AFADEE7E3B20124009201940A00A4
:1041E000310006F03BFF0500D4E70825D2E70125A2
:1041F000D0E70B25CEE70D25CCE7C046F3FF000046
:10420000F4FF000002290000D661FF1FAC61FF1F10
:104210004862FF1F332310B5040003700A220749C8
:10422000013006F099FF064B0F201B681A0AE37253
:1042300022731A0C1B0E6273A37310BD0862FF1F5A
:104240003862FF1F30B5012503790400BFB02B424F
:1042500013D00B49408806F06DFA28420DD06A460B
:10426000084B02A81B889380FFF7D4FF6B46D880C9
:104270000022608801A903F069FB3FB030BDC04651
:10428000CE61FF1F7E41FF1F10B5024804F0E0F928
:1042900010BDC0464542001170B5160004AA14882E
:1042A00005AA15784A685078117800022A4A08430E
:1042B000801805284BD807F0A7F903131E29343FAF
:1042C0000720022C0BD80322121BAA4200D92A0075
:1042D00022491A803000091906F03EFF002070BD07
:1042E0000720112CFBD81222121BAA4200D92A0047
:1042F0001B491A80EEE707200E2CF0D80F22121B64
:10430000AA4200D92A0017491A80E3E70720032CA4
:10431000E5D80422121BAA4200D92A0012491A80A9
:10432000D8E70720032CDAD80422121BAA4200D9AE
:104330002A000E491A80CDE70720022CCFD803228D
:10434000121BAA4200D92A0009491A80C2E700229A
:104350000A201A80C3E7C046DCD5FFFF46B800112B
:10436000F461FF1F36B8001131B800112CB80011EC
:1043700028B8001110B50D21024A034806F052F981
:1043800010BDC0461CB800119441FF1F10B5084C69
:10439000E368002B08D18022064B52021B689B1851
:1043A0006360054B1B68236007F06EF8A06010BDCA
:1043B0003862FF1FC8F00040CCF0004070B5184ACA
:1043C000936A916A9942FBD116498A689A421FD32F
:1043D0009A1A8B60144B0126186893B2D202D20E3F
:1043E0004343424300204C681B0A1B1912029B18CE
:1043F0000E4C0A684B60551CA3420CD8002801D013
:104400004B600A600A4A136008680A4B186070BD66
:10441000581E821ADDE7084A30009B182A00EAE796
:1044200000F000403862FF1F140AFF1F40420F00D7
:10443000C8F00040CCF00040C0BDF0FF70B51F4C8C
:1044400023793F2B01D93F2323711D4B22791A7009
:104450001878C0B207F0F8F818231A491A4A0B80E6
:104460001A4913800B805380A379194980200B804F
:104470000C21938001334B43164D191C00018342DC
:1044800000D9011C2980D1806379002B01D101332F
:104490006371237A012B01D8022323726279237A74
:1044A0000D4853430A21584307F036F80B4D286056
:1044B000E379052B01D81023E37170BD2C62FF1F37
:1044C000480AFF1F7E42FF1FCC43FF1F7C42FF1F95
:1044D0007A42FF1F7842FF1F710200001462FF1F23
:1044E00070B520210020FEF701FF0C4C002805D1FB
:1044F0000B4B23CB23C4FFF7A1FF70BD0C22200080
:104500000849FEF7C7FE0C2802D0054B23CB23C475
:104510001C2205490548FEF7BDFEECE72C62FF1F93
:1045200064B80011FC0C0000D1F100008961FF1F8C
:10453000F0B51D4C8022A544040088206946520134
:10454000400507F021F8902212016A441300200070
:1045500032C832C316C816C38023144C144FA66841
:104560009B033343A3603B6006F016FE8823A068DC
:104570005B05C01806F000FE002588232900802274
:10458000A0685B05C01840196944520006F03CFF62
:1045900080230135FF355B019D42EED1A6603E6070
:1045A000044B9D44F0BDC046FCEFFFFF3C43FF1FA2
:1045B0009808FF1F04100000F0B5040087B0002821
:1045C00025D0684606F0F8FD1B4C022806D10622CD
:1045D0006946200006F0E0FF002816D06946002357
:1045E00001250F262F00E25C0133100910308740AF
:1045F00038002F00324097403A0002434A610439A4
:10460000062BEFD16846FFF793FF07B0F0BD1822E5
:1046100069460A4806F0B8FF6A46A300D35801333A
:1046200005D01822FF21684606F0E6FFEAE70134CC
:10463000062CF1D1E9E7C0466509FF1F000900110A
:10464000F0B5002704000E00150085B0BA4200D175
:1046500090E04A1C0B7801924A788978090211434C
:10466000F27812040A43317903700906114300916C
:1046700003914770192B30D80F2B1ED8062B00D171
:1046800046E1072B00D13CE1BB426ED0012B2FD17C
:10469000BC4AAB1E0092132B07D87378002B00D0B6
:1046A000C1E100F0A9FA00F0DFFAB74B00991F78DA
:1046B000601C7A1E06F050FD5CE0180010380928D6
:1046C000E4D807F041F88901A901E3FFE3FFE3FF24
:1046D000E3FFE3FFE3FF7A00A200562B67D022D866
:1046E000332B00D137E1552B47D0232B00D136E1B6
:1046F000DB2B00D0A3E1042D00D882E01027052D8C
:1047000005D06F1F3A000098711D06F025FD0522A7
:104710003100200006F020FD3A000099601D06F0EF
:104720001BFD053726E0712B00D1F8E0722B00D17C
:1047300008E1DC2BDCD1022D63D973784370B378A8
:1047400083706B461F88032D05D0033D3900AAB244
:10475000F01CFEF7D9FC39001022E01CFEF79AFD90
:10476000C71C002806DA60704DE00C22874906F06D
:10477000F3FC0C27380005B0F0BD6A1E844D0C2AEE
:1047800013D8002A0AD02800019906F0E5FCFFF7AB
:1047900055FE0C2228007F49FEF7B6FC0C222900AA
:1047A000601C06F0D9FC0D27E4E70C22EBE7784DFE
:1047B000794B2A0043CB43C2E9E7784E112D12D141
:1047C00010223000019906F0E7FE00280BD01022DD
:1047D0000199300006F0C0FC102271493000FEF74C
:1047E00093FCFFF7E5FA102230006D49FEF752FD09
:1047F0000200102805D13100601C06F0ADFC112725
:10480000B8E7FF2363700227B4E7102D53D1777800
:10481000032F0DD1634D0E22B11C280006F09CFC25
:104820000E222900A01C06F097FC67701027A1E754
:10483000042FE6D15C4DB11C0E22280006F08CFC42
:1048400029000E22A01C06F087FC564D574E1C2254
:104850002900300006F0A0FE002829D01C222900E3
:10486000300006F079FC1C2230005149FEF74CFC68
:1048700040232A785B421343290028002B7000F064
:1048800023FA4C4E06222900300006F085FE00284F
:104890000ED006222900300006F05EFC06224649B2
:1048A0003000FEF731FC0123444A51780B4353702A
:1048B00004236370BAE7022DA3D17678012E10D1BC
:1048C0003A4D1C2228003A49FEF7E4FC1C2806D188
:1048D0000E222900A01C06F03FFC6670A6E7FE230E
:1048E00090E7022E8DD11C2230483149FEF7D2FCD0
:1048F0001C28F4D10E223249A01C06F02DFC657054
:1049000094E712222F49013006F026FC132731E7E5
:1049100008222D49013006F01FFC09272AE7012D46
:104920000CD07178F02900D96BE7284D288801F068
:10493000AFFB274B2A885200D35A63E7234A244B04
:104940001288F8E71D4B012D03D072785A7042701F
:1049500059E75B7856E7FFF75DFC07000AE7042D8F
:1049600005D91C4D009B2B6006F08EFDA860FFF75B
:1049700025FD0422039003A9601C06F0EDFB05272A
:10498000F8E6C0462964FF1F2764FF1F70B80011B6
:104990002C62FF1FFC0C000064B800115061FF1F67
:1049A0000DBC00006D61FF1F7B61FF1F8961FF1F50
:1049B000D1F100006509FF1FADAC00002862FF1FA8
:1049C0009761FF1FF461FF1F4043FF1F8042FF1FDD
:1049D0008464FF1F3862FF1F2A4E062D15D9062258
:1049E0003000019906F0D8FD00280ED0062201996A
:1049F000300006F0B1FB062223493000FEF784FBAD
:104A00000123224A51780B43537006223100601C67
:104A100006F0A2FB0727ADE6012D00D1F1E6707884
:104A2000FFF7CAFDEFE6013D2A000199009806F064
:104A300093FB17490098AAB2FEF766FB33E6DA2B20
:104A400000D0DEE6042D00D8DBE6082D17D9B379B7
:104A500072791B021343F27912041A43337A1B064C
:104A60001343009A1360009B05221B68310020004D
:104A7000039306F071FB0422601D03A94BE7FE239C
:104A80006370F0E76509FF1FADAC00002862FF1FEF
:104A9000AEDE000070470000020010B5094B0A327C
:104AA000094C92B2DA815A8298811882207802F0F9
:104AB00055F90422054B012120781A7006F024FED6
:104AC00010BDC046CA42FF1F7264FF1F7164FF1F02
:104AD000013870B5042809D806F096FD03092708A7
:104AE0001200204B0221187806F00EFE70BD1D4BFF
:104AF0000821187806F0B0FC00221B4B1A74F5E769
:104B000080220024184B52001A82FA22DC74174BC0
:104B1000144D5B7A920008215A43287806F08CFDE8
:104B20002100287806F0B0FBE0E70E4B082118784A
:104B300006F092FC0E48FFF7BBF90C4B0D4A9B792F
:104B400093800D4A13800022074BDA740132FF3242
:104B50001A820A4B5B78002BC8D0094A136006F012
:104B600033FBC3E74862FF1F1462FF1F2C62FF1F65
:104B70008942FF1FCC43FF1F7A42FF1F2862FF1F9D
:104B800034F0004010B5002909D1092807D10638B2
:104B900005F018FA024B8021187806F0B5FD10BD1B
:104BA0004862FF1F10B5012909D1092807D106382D
:104BB00005F008FA024B8021187806F0A5FD10BD1B
:104BC0004862FF1F0300F0B50A4D8E18B14202D1B2
:104BD00052008018F0BD0C782F6824093C5D0F2727
:104BE0001C700C7801313C402F683C5D5C700233D6
:104BF000ECE7C0467442FF1F0C22124B10B51A702E
:104C00000B23114C11492370093A023B1048637081
:104C100006F0A2FA2D2301220E490F486371FFF717
:104C2000D1FF01220D49FFF7CDFF01220C49FFF70B
:104C3000C9FF030000200B4902001870FEF764FA58
:104C400010BDC0464664FF1F2764FF1F46B8001111
:104C50002964FF1F6709FF1F2D64FF1F6609FF1FDF
:104C60006509FF1FAEDE000070B5134C1422200052
:104C70001249FEF70FFB431E114D132B19D8AB78C9
:104C8000002B16D0431C2B7009236B7000230019D6
:104C9000037028780B4B01302900C0B2187006F061
:104CA000DBFC297822000139C9B2002005F0D8FBCD
:104CB00070BDFFF7A1FFECE72964FF1FAEDE000027
:104CC0002764FF1F4664FF1FF0B54A784F790E79BD
:104CD000CD788C780B78077046708570C47002713F
:104CE0004371F0BD10B5114B1A781870002A0ED020
:104CF00000280BD10E4B1A78062A07D85423D3402C
:104D0000DB0703D50B4B187802F028F810BD0028FC
:104D1000FCD0074B1B78012B02D0033B022BF5D8AC
:104D2000044B0121187806F0EFFCEFE74A64FF1FFF
:104D30007164FF1F7264FF1FF7B5574D574A5849FA
:104D40002870092005F018FA0121032005F03AF92E
:104D5000032005F0FFF906F09FFB0322514952485A
:104D6000FFF730FF2D24030088211C700422490521
:104D70000130FFF727FF302304704C4E4C4C43703A
:104D800083702E3B062230004A49E387FEF782FA01
:104D9000062813D0300006F00FFA022809D00321AC
:104DA000300006F0D1F98D23F3706E3B3371193367
:104DB0007371062230003F49FEF7A6F93E4B1B688F
:104DC000FC335E64FFF750FFFEF7F2FF0020FFF7B1
:104DD00089FF3A4E80223168394F08000197394BDC
:104DE000394F104011424FD07D3A01981A70FFF7A9
:104DF000A7F838703A78354F01213878019B01F0D7
:104E00006FFF334A334B12783878002101F068FF86
:104E10000122314B314F1A70314B9B78552B35D1D4
:104E2000193B7B742F4A304BA381E281238262823B
:104E30002021287806F038FA0120404205F05CFB7A
:104E40000120404205F0F8FBFFF794FAFEF7B0FEB0
:104E500001204042FFF720F9012006F085FBF020F9
:104E600001F0FAF80121287806F04EFC287802F0CB
:104E7000D1F81E4806F000FCFEF740FD1C4B1D4A11
:104E80009B689B18BB60F7BD1870B3E76422737909
:104E900053431A000A32C7E74862FF1F854B0011CF
:104EA000A54B00114043FF1FF461FF1F6509FF1F61
:104EB000CA42FF1FADAC00008064FF1F2C62FF1FC1
:104EC0008942FF1F2664FF1FA842FF1F7264FF1F55
:104ED0004664FF1F2764FF1F1864FF1F1462FF1F33
:104EE0002862FF1FCE090000C40900004A62FF1FAC
:104EF0003862FF1F0000B8FCF8B50A0020230D003F
:104F00001A40194200D17EE0834B1B78002B50D011
:104F1000FFF754FA814B824C824E99686268737A2B
:104F20008A1ADB039A4247D36160FEF7E7FC637C91
:104F3000002B3BD0013BDBB26374002B36D17A4BA4
:104F40009B78552B01D106F03FF9E37C774F002B7E
:104F500045D00021032005F035F8F3796374BB7860
:104F6000002B23D1A27C002A02D0A374FEF75CFDA3
:104F70000121052005F026F83B880021013305209A
:104F80003B8005F01FF86A4E3000FEF791FF3100BC
:104F900006F03AF90121052005F014F8002105205A
:104FA000E17405F00FF8C820FFF776FD237C01338C
:104FB000237420206840F8BDA37C002BB7D00023C9
:104FC000A374FEF731FD594A594F13883800013355
:104FD0001380FEF76DFF390006F016F9A7E7A27CF3
:104FE000002A02D0A374FEF71FFD3B8801333B80EB
:104FF0004F4F3800FEF75CFF390006F005F96423D7
:1050000070795843D0E70BB2002B0ADA494B187875
:1050100006F0F2F9002801D006F056F980200002CF
:10502000C8E70224214206D03D4B01201A74FFF745
:1050300059FE2000BEE70824214204D0FFF7BEF944
:10504000FEF75CFCF5E710230E001E4019420FD05E
:10505000FEF7EAFC304B1B78002B07D1FEF7BCFDB6
:10506000304B1B68DB0701D5FFF70EF91020A1E7D5
:105070000124214209D0304800F0AEF806F0FCF8D7
:105080003100032004F09EFFD3E70B063BD5092037
:1050900004F074FE254B5A7A002828D0224203D00F
:1050A00022435A72802085E71D4922435A721A4AC8
:1050B000C86812780130C8609C701A48002A1AD05B
:1050C0001A881B4C01321A800123CB74C3791B4A06
:1050D0004B74124B20009B689B188B60FEF7E8FE18
:1050E000210006F091F8C820FFF7D6FCDAE7A243CA
:1050F0005A729870D6E70368DB07D3D5FFF75EF9DD
:10510000FFF7C2F8CEE7042408002040214200D176
:1051100051E7FEF7DDFF8CE74A64FF1F3862FF1F8F
:105120001462FF1F2C62FF1F2862FF1F0862FF1F0F
:105130008942FF1F4862FF1F6C42FF1F000082FC74
:10514000F0B51B4B1B4F1B883A8804001A4E1B4DB1
:1051500085B09A420DD832889A420AD3184B1A88E1
:105160002B889A4205D1174A174B12881B889A42FE
:105170001BD0052000F0C6FF3B8802AA13803388AD
:10518000019053802B88114D93800F4B02A91B88EF
:10519000D3800F4B2A78188802F0E2FC0D4B0821CF
:1051A0002878019A1C7006F0D7FA05B0F0BDC04609
:1051B0001664FF1F7E42FF1F7C42FF1F7A42FF1FC3
:1051C0001464FF1F1264FF1F7842FF1F7264FF1FE9
:1051D0008042FF1F1064FF1F13B50C4B1C78002C7E
:1051E00011D1002801D00A4B18600A4A0A4B1178E5
:1051F0000A4A10780A4A01920A4A0092002205F0EF
:1052000027F8200016BD1124FBE7C0467164FF1F7C
:105210000C64FF1F7064FF1F6064FF1F7264FF1F38
:105220004C64FF1F5064FF1F10B5064B12201B7803
:10523000052B06D1044B13221988044B187801F072
:105240003DF910BD7164FF1F8042FF1F7264FF1F94
:1052500010B500240122114B52421870104B1C70E3
:10526000104B1A8001F0D6FE04220F4B21001A7059
:105270000E480C3206F060F8102221000C4806F0AF
:105280005BF807220B4B1C600B4B1C700B4B1C700C
:105290000B4B1A700B4B1C7010BDC0467264FF1F85
:1052A0007164FF1F8042FF1F7064FF1F6064FF1F57
:1052B0005064FF1F4C64FF1F2664FF1F2564FF1FFF
:1052C0008242FF1F2464FF1FF8B5174C06002578A3
:1052D00006A814240078052D23D1B41F134FA5B2BE
:1052E0001824BD421DD88D1FADB2BD4219D8FA2574
:1052F0006D00AA4215D21D000D4F0A3DADB2BD4250
:105300000FD80C4C26800C4C21800C4900240A80BC
:105310000B4A1380FFF714FF0A4B0421187806F09C
:105320009BF82000F8BDC0467164FF1F790C000097
:10533000750C00007E42FF1F7C42FF1F7A42FF1F58
:105340007842FF1F7264FF1FF0B50BB20D0089B0E9
:10535000002B00DB70E1A44E307806F04DF8041EFF
:1053600050D00378A22B00D122E1D02B1AD0912B60
:1053700045D143780E2B42D19C4B82889A423ED134
:105380009B4A83681278052A39D1032018567F2852
:1053900035D0984B1B68002B31D05B68002B2ED08A
:1053A00098472CE08078072829D806F02DF90428A2
:1053B000183F3F74A8D86378002B0CD101218C4B87
:1053C00019708D4B1A78002A5BD08C4B307801F025
:1053D00087FC002855D00722854B1A7051E0617870
:1053E0000029F8D1E378002B11D0854A854B12783B
:1053F000307801F075FC60706378002BEBD12000F1
:1054000005F062FF80200002684009B0F0BD784BD3
:105410001B78022BF3D00121307806F015F8002814
:10542000EAD10121307806F06FF9E5E76378002BC7
:10543000D1D16F4F032807D13B78052B02D101331F
:105440003B701EE00223FBE76F4B1A886F4B029301
:10545000002A0BD01B78002B03D00121307806F0F6
:105460007BF93B78062B04D1013BE9E7029B1A70DC
:10547000F7E7042B41D10121029B3078197006F027
:1054800043F95C4B1B68002BB9D01B68002BB6D0CE
:10549000574A107884E76378554F002B27D10622AE
:1054A000211D5B4805F058FE62895A4B5A491A8003
:1054B000A2895A4B1A80E3890B800521397058491B
:1054C0000A80584A1380228A574B1A80574B1B7800
:1054D000012B09D11F2000F015FEFA229200424351
:1054E0000421307806F038F90022484B75E7312B5B
:1054F00000D070E70022454B1A700323A0E7062274
:105500000021434805F018FF0023454A0421138079
:10551000444A30781380444A138005F09DFF0821E7
:10552000307805F099FFA379083B5A425341304A3D
:1055300003331370304B1B78002B06D0334B30787D
:105540001A78002A06D001F009FC0122314B5242A0
:105550001A8096E70121197006F0D6F8F5E70821C0
:10556000307805F079FF6378002B00D047E72C4BAB
:105570002D4F0293E388029A04211380294B30783F
:1055800003932389039A138063893B8005F05CFFB2
:10559000002800D033E7264B1B68002B00D12EE7F4
:1055A000039902983A88098800881B68984726E77B
:1055B0004379132B00D022E70389012B0AD11D4B1D
:1055C0001B78022B06D10821307805F045FFFFF744
:1055D0002BFE14E7052000F095FD0821020030782D
:1055E00006F0BAF80BE7C0467264FF1F051400000E
:1055F0007164FF1F0C64FF1FA842FF1F8942FF1F39
:105600004664FF1F2764FF1F4864FF1F4A64FF1F93
:105610001964FF1F8042FF1F2064FF1F2264FF1FC9
:105620001664FF1F1464FF1F1264FF1F1864FF1F1E
:105630000864FF1F1064FF1F8020C001014200D0DA
:10564000E2E6CB0731D5324B1B78002B1DD0314E13
:1056500005AC3378052B1AD1023B23702E4B210069
:105660001B7823722D4B1B7863722D4B187801F039
:10567000DBFA002809D007202A4B30701B68002B6A
:1056800003D01B68002B00D098470120BCE60E20F9
:10569000254B06221B7825492370254B1B78637008
:1056A00002ABC01805F058FDD8E7022308001840E7
:1056B000194209D0174B1B78052B03D11D4B1888B5
:1056C00005F082FF02209FE60424214203D0FFF769
:1056D00037FD200098E6082308001840194200D141
:1056E00093E6154B1C78012C03D0022C0DD008201A
:1056F0008AE6124B124A134913481B8812880988FC
:1057000000880094FFF7E0FDF1E7FFF78DFDEEE77D
:105710004A64FF1F7164FF1F8242FF1F2464FF1F42
:105720007264FF1F0C64FF1F2664FF1F8342FF1F6C
:105730002564FF1F8042FF1F1064FF1F7842FF1F78
:105740007A42FF1F7C42FF1F7E42FF1F0200F0B51E
:1057500001270A480A4E51188B1A002B00DCF0BDB5
:10576000082415784308684038404000805B013CBD
:1057700058406D08002CF5D10132EDE7FFFF000025
:105780008EB80011F0B500250F269D4200DBF0BD5C
:105790004C5D070944403440A400A05801357840CE
:1057A000F3E70000F0B589B06A460D000B000F2743
:1057B000110010351C780133260024093E40167074
:1057C00054700232AB42F5D12023024AFFF7DAFFD0
:1057D00009B0F0BD94B80011F0B54E780B7889B0DF
:1057E00036020C00170001901E43012A61D9954B27
:1057F0009E4200D877E001339E421CD1062A17D181
:10580000CA788B7812021A430B791B0413434A7926
:1058100012061A438C4B5A6100221A705A808B4A26
:105820005A608B4A9A608B4ADA60002009B0F0BD5A
:1058300088225205EEE7884B9E423CD182498B7804
:10584000002B00D0F6E00C2A31D10F22A37893432D
:10585000E27812021343227912041343627912068A
:1058600013434B60E279A07912020243207A0004CC
:105870001043627A12060243CA60E27AA07A1202E8
:10588000024376484A81834208D804236E49142291
:1058900001980B7005F060FC1420C7E71201D218C4
:1058A00089235B059A42F0D801238B70BDE7022A59
:1058B000FAD00523EAE76A4A01239642E6D1FFF7C8
:1058C000B3FC052F0CD9E378A2781B02134322798D
:1058D00012041A4363791B061343624A039313604D
:1058E00005F072FCA1E7584D2B78002B9DD1AB78C9
:1058F000002B00D1A0E02B8901339BB20093B3426F
:1059000000D091E0132AD4D9CF7C8B7C3F021221A6
:1059100020001F43FFF71AFF874200D08EE0002EC1
:105920003DD1E378A2781B0213432279E96812047F
:105930001A4363791B06134303930A228B4212D145
:10594000FF23A370E370237163716B89002B09D16E
:10595000E37B227C1B0212041343A27B13431B092B
:1059600001336B8100226B89002B8ED0002A67D116
:10597000686837013818000B6B6900030390984280
:1059800005D9686105F0F8FBEB780133EB706868C6
:105990001022A11C381805F037FD2E8145E76F89CC
:1059A000009A7B1E9BB293423AD1E278A37812020E
:1059B0001A43237905A81B04134362796C68120605
:1059C0001A43EB6800920392211D0C22049305F008
:1059D000C3FB0120260004A940421036FFF7E2FE77
:1059E000013F012F17D1009A0B232861824200D07A
:1059F0004CE704221C49200005F006FD042203A9FF
:105A0000686805F0C1FDE968039AFF23914200D15F
:105A10003CE7F73B3AE73100FFF7C4FE1036DFE71B
:105A20000923B742A4D831E7009BB34200D9FCE672
:105A300007232BE7022329E7032327E7062325E78C
:105A40000A2323E7FFFE0000AC42FF1F0000011104
:105A5000FFFF00005048593601FF0000FFFF001112
:105A600002FF000034F00040B842FF1F10B5034CA5
:105A70000B000122210000F06BFA10BD2D5C00111B
:105A80000B8870B506000D000224162B11D92B00CF
:105A90000322094900F05CFA041E0AD1074B2A8848
:105AA0001B88191C934200D9111C300089B200F0E8
:105AB000EFFA200070BDC046595C00118664FF1FDC
:105AC00010B54A780400013A0B000220012A07D8D9
:105AD0000A78002A04D005222000024900F038FA92
:105AE00010BDC046875C00110A7810B50B00040099
:105AF0000220002A04D007222000024900F028FAE0
:105B000010BDC046335D00110A7810B50B000400CB
:105B10000220002A04D009222000024900F018FACD
:105B200010BDC046995D001110B5034C0B000B224F
:105B3000210000F00DFA10BDC95D001110B5034C35
:105B40000B000D22210000F003FA10BD3B5E001196
:105B500010B5034C0B000F22210000F0F9F910BD25
:105B6000955E00110A7810B50B0004000220002A8F
:105B700004D011222000024900F0EAF910BDC0460D
:105B8000A55E0011002310B51322190000F0E0F902
:105B900010BD000010B5034C0B001722210000F0CF
:105BA000D7F910BDF75E0011002310B519221900B6
:105BB00000F0CEF910BD000010B5034C0B001B2205
:105BC000210000F0C5F910BD315F0011F7B58489DF
:105BD0000D0006000121002C22D000238268D3563C
:105BE0001778002B1EDA0C2C1AD90C3CA4B213190E
:105BF00040880093230002F086FE431E9841013046
:105C00007B06DB0F6B703F23013C1F40A4B2287062
:105C1000AF70AC80002C07D0B3680133AB600021BB
:105C20000800FEBD0020EBE7AC60F8E70B780370DE
:105C30004B8843704B881B0A83700B79C370042018
:105C400070470420022B06D10020537811781B02E4
:105C5000009A0B43138070470B8803700B881B0A54
:105C60004370022070470420009983420AD1537880
:105C700010781B0203430B80D37890781B020343F8
:105C800000204B807047F8B50D004B7801240021AF
:105C9000461C03702B788B4201D82000F8BD6B782E
:105CA000B01C4F1C012B10D1890069184B880222AF
:105CB00033704B88B9001B0A7370691805F024FC17
:105CC00004360434A4B2F9B2E4E7122359436B1842
:105CD0005A88043132705B8810221B0A737069186D
:105CE00005F012FC12361234ECE770B5049D140076
:105CF0001E00052B01D8042070BD637812781B02AA
:105D000013432B80E378A2781B02134302226B809B
:105D10002A71211D681D063E05F0F6FBB2B22A81EC
:105D2000E92AE8D82800A11D0A3005F0EDFB002083
:105D3000E2E7002310B50A789A4201D8900010BD1E
:105D40009A008A185488013304705488DBB2240AFC
:105D50004470948884709288120AC2700430EAE712
:105D600010B51100029C062B04D004201022142B25
:105D700001D010BD022222714B7808781B02034328
:105D80002380CB7888781B02034363800431601D35
:105D900005F0BAFB0020ECE710B50C788B780431E5
:105DA0005C43E4B203702200013005F0ADFB601CDF
:105DB00010BD0420022B06D10020537811781B025D
:105DC000009A0B431380704710B50C000A8802310B
:105DD00005F09AFB208810BD70B504000D000498F2
:105DE0001100012B01D8042070BD167852781202E0
:105DF000324302800200F13255701470E125002C0C
:105E000000D10C35023B9AB24280AA42EBD8023153
:105E1000043005F079FB0020E6E704200099834276
:105E20000AD1537810781B0203430B80D378907803
:105E30001B02034300204B80704710B50C000A88FA
:105E4000023105F061FB208810BD000070B5012112
:105E50001E000420049C0E400B4218D1CB40DDB242
:105E60008D4214D90A49DBB2098899420FD3230025
:105E7000EE331D703300580011184978165C090282
:105E8000314301332152D9B28D42F4D8002070BD84
:105E9000C442FF1F10B50C000A88023105F034FB24
:105EA000208810BD10B50C788B7804315C43E4B2C7
:105EB00003702200013005F027FB601C10BD10B5F7
:105EC00011000298032B01D8042010BD14785278D9
:105ED000043B120222430280CA788C7812022243C9
:105EE00042809AB28280EB2AEED80431063005F067
:105EF0000BFB0020E9E710B50C000B8803700B8842
:105F00001B0A43704B8883704B881B0AC3708A88B6
:105F10000430063105F0F8FAA088043080B210BDD4
:105F20000420012B03D100201378009A13707047CE
:105F300010B50C000B8803700B881B0A43704A884D
:105F40000230043105F0E0FA6088023080B210BD02
:105F5000F0B589B003931E4B029242000700D05A5D
:105F6000019102F020F81325061E2DD0029B01247A
:105F70000370019B002B04D0001903999847001966
:105F800084B26B461B7A5BB2002B0FDA102138000B
:105F900002F01CFB1925002813D130003219E1B2A0
:105FA00002F066FC051E0CD10C34A4B2042304AA32
:105FB000380005A993800696948101F0AFFD051E77
:105FC00002D0300005F068FB280009B0F0BDC046E3
:105FD0008464FF1F70B505000C0000280CD0002061
:105FE000814209D010222000044905F08DFA0120D9
:105FF0002B7823736B78637370BDC046D4B80011DF
:10600000F0B506000D0017001C0085B002291BD05A
:106010000020102907D1022B07D0102B03D115E047
:106020000020102C08D005B0F0BD69463800FFF7FD
:10603000D1FF2A0069460BE069463000FFF7CAFF2E
:1060400022006946380004E0022BE9D12A00390019
:10605000300005F0E1F8E6E7031CF02800D9F02352
:10606000032008499AB2013A0B80D317034006492E
:106070009B189B100B80D30F04499B185B100B805F
:106080007047C046C842FF1FC642FF1FC442FF1FE1
:10609000034B1B888B4202D3024B4000C152704716
:1060A000C842FF1F8464FF1F014B4000185A70470D
:1060B0008464FF1F1722014B1A8070478464FF1FFE
:1060C00070B505000E2005F00FF9041E13D0D02383
:1060D000037000230622837007494570033005F0E2
:1060E00013FA064B2100DA8A62811B7E2373044B6C
:1060F000187805F021FB70BDA064FF1F9064FF1F9E
:106100001843FF1F262803D8024B4000C05A70478F
:106110000148FCE7CA42FF1FFFFF000070B5060000
:106120000C00094D1C220021280005F005F9074B41
:106130001E70074B1C7005F0DFF90123002801D009
:10614000002312202B7070BD9064FF1F1843FF1FA7
:10615000B164FF1F70B505000D4C0800E260A1603E
:1061600010220021656005F00FFB012803D11021EA
:10617000A06802F058FD10220021280005F004FB61
:10618000012803D11021606802F04DFD70BDC046AA
:106190009064FF1F70B5041E05D1002903D00622AC
:1061A0000D4805F0B1F90D4B1D78012D11D1002CD2
:1061B00005D102221A7004F0BFFF280070BD002232
:1061C0001A70074B1B78FF2BF7D02000FFF778FFE2
:1061D000F3E70025F1E7C046A064FF1F9064FF1FAE
:1061E0001843FF1F030010B5002801D1002010BD87
:1061F00000780B4A002803D15988D1821B79137685
:106200001378022BF2D10023984200D1033313708C
:10621000044B1B78FF2B01D0FFF752FF0120E6E76C
:106220009064FF1F1843FF1F002911D000280CD0D5
:106230004B79012803D140225242134303E03F220D
:106240001340032802D001204B7170474022F4E72D
:106250000800FAE770B5094D0100287800280BD036
:10626000074C0622200005F04FF921002878FFF79F
:10627000DBFF200005F060F970BDC046B064FF1F71
:106280008A64FF1F00290AD0012808D13F224B79D8
:106290009343C02B03D0403B5A425341981C704754
:1062A00070B5174D06002B78FF2B15D00A2005F08E
:1062B0001BF8041E10D0D0230370C83B8370114B11
:1062C00011491B784670C3700622043005F01CF992
:1062D0002100287805F030FA0C4B1B78012B0DD1EA
:1062E0000B4B1B68002B03D09B68002B00D09847FA
:1062F000084B04211878084A05F09EF970BDC04685
:106300001843FF1FB064FF1F8A64FF1FAC64FF1FA8
:10631000D864FF1FDC64FF1F60EA0000014B98682F
:106320007047C0469064FF1F014BDB6818687047D8
:106330009064FF1F074B10B5DA68136801331360D0
:10634000054B1878FF2803D08021C90105F0DCF93E
:1063500010BDC0469064FF1F1843FF1FF7B50E0025
:1063600002F0C8F8051E1CD00E4B06621F78002FE5
:1063700000D10778AB791020019304F0B5FF041E1B
:106380000FD0D0230380C73B8370019BE91DC370EE
:106390000622043005F0B8F821003800E66005F068
:1063A000CBF9F7BD1643FF1F014B18787047C04665
:1063B000B064FF1F054B002805D1054B1A78054B2B
:1063C000002A00D1014B18007047C046A064FF1F8F
:1063D000B064FF1F8A64FF1F014B58687047C046B6
:1063E0009064FF1F024B1868431E9841C0B270476B
:1063F000B464FF1F421E03000120152A03D9FF3B8E
:106400005A425341D8B27047F0B51C0000230E0029
:1064100085B0039002920B70029A934201D3002040
:1064200019E0E55C5A1CD2B2002DF8D0029851193F
:106430008142F4DC0233DFB2A35C18000193FFF762
:10644000D9FF002807D0013D019A0399EBB23370C0
:106450008A4202D1E01905B0F0BDDB19DBB2DBE7FF
:1064600010B50C0002F09EF803001220002B03D0A0
:106470002100588805F068F810BD000070B50E4D79
:1064800084006359002B15D0186A002801D005F04C
:106490000BF92B59586A002801D005F005F92B5942
:1064A000986A002801D005F0FFF8285905F0FCF89B
:1064B00000232B5170BDC046C064FF1F1C4B70B53C
:1064C00004000E00150099420AD11A4B1B68002BDC
:1064D00001D1122070BD1B68002BFAD09847F9E754
:1064E000154B994215D1134B1B68002B0AD01B6822
:1064F000002B07D09847002804D1104B1C70104B7C
:106500001D70E7E729002000FFF7AAFF0028E1D16E
:10651000F3E7080001F0EEFF0028DAD0037803204B
:10652000A342D7D12900300005F00EF8D2E7C046CB
:10653000FEFF0000BC64FF1FFFFF0000B964FF1FE7
:10654000B864FF1FF7B50400808801F0D3FF002571
:10655000A84203D00578A08802F008F81C4E3378D2
:10656000002B1FD0AB421DD11A4B28001978FFF722
:1065700077FF002818D000233370A3790820A7786C
:10658000A688019304F0B0FE011E0DD0D023037045
:10659000CA3B8370019B477086808371280005F099
:1065A000CBF801E0002DE8D1A0880B4B8200D35836
:1065B000002B01D0FFF762FF1721A088FFF768FDCD
:1065C000A08801F027FDA08801F0FEFDF7BDC046C0
:1065D000B964FF1FB864FF1FC064FF1FF0B587B028
:1065E0001D000CAB1B88070001930DAB1B8814200A
:1065F00002930EAB1B88160003930FAB1B88009110
:10660000049310AB1B88059304F06EFE041E1AD091
:10661000D0230370CB3B47708370C67006222900DD
:106620000430002D11D004F06FFF019B2100638125
:10663000029B0098A381039BE381049B2382059B1B
:10664000A37405F079F807B0F0BD04F075FEECE72F
:10665000F7B5009308AB1B8807000C200D0016004F
:10666000019304F041FE041E13D0280001F042FF04
:1066700000280FD00078D0232370C93BA370009B63
:1066800021002381019B6770A580E680638105F06E
:1066900053F8F7BD014B1878EDE7C0461843FF1FCC
:1066A00013B5040064890389C2888188C078009486
:1066B000FFF7CEFF13BD000010B5044C2068002882
:1066C00003D004F0F1FF0023236010BDC464FF1F5A
:1066D000A122F0B5818892004A43384B384F1B689D
:1066E00004009B189D2292009B18827989B01A6041
:1066F0003B68002B5FD01D78324B1B68002B04D009
:106700005B68002B01D00020984726000836310036
:10671000E079FFF7B7FD237DE0710200E078049394
:10672000638A29000393238A0293E3890193A38850
:1067300000933300FFF752FFE378002B0BD1E2897F
:10674000A379A18802920196E279280000920122A1
:1067500001F0DAFEE0703B68002B20D0FFF7ACFFC1
:10676000194D287800281AD0184B1978FFF778FEB1
:10677000002814D02B78E67808200793A78804F027
:10678000B3FD011E09D0D0230370CA3B467083704D
:1067900087808671079804F0CFFF00232B701721A4
:1067A000A088FFF775FCA08801F034FCA08801F0F8
:1067B0000BFD09B0F0BD064B9DE7C0463409FF1F35
:1067C000C464FF1FD864FF1FB964FF1FB864FF1FB4
:1067D0001843FF1FF8B5070008000E0001F08AFEFD
:1067E000041E18D02620FFF78DFC051E00D1257849
:1067F000062004F079FD041E0DD00021062204F0CD
:106800009BFDD0232370C23B21006770A370A6803C
:10681000E8B204F091FFF8BDF0B585B001930AAB82
:106820001B78070002930BAB1B7808000D00009249
:10683000039301F05FFE061E22D0102004F054FDE9
:10684000041E1DD01022002104F076FD2620FFF743
:1068500059FC002800D13078D0232370C13BA370AD
:10686000009B21002372019B67706372029BA580CD
:10687000A372039BC0B2E3720C9BE36004F05CFF65
:1068800005B0F0BDF7B50D00019001F033FE071E15
:1068900020D00E2004F028FD041E1BD02620FFF778
:1068A00031FC061E00D13E78D0232380C53B062252
:1068B000A370F91DE01C04F027FE019B2A006381F0
:1068C0000123DD401A401D40210022736573F0B2A0
:1068D00004F032FFF7BD0000F0B585B00290100063
:1068E0000D0017000A9E039301F004FE041E31D030
:1068F000029B002B2ED1039B02795B0724D5122328
:1069000013430422002E08D10B99002905D10C99BC
:10691000002902D10D9900291AD01A430D9B22712A
:10692000002B00D0C9E0002E00D1CFE0002D00D018
:10693000CCE0606A002801D004F0B6FE1C213000D3
:1069400004F002FD606205E002239A430E33D7E7AC
:1069500093432371654BBA00D458002C00D1AAE0B0
:10696000002E10D0236A002B03D11C2004F0F4FD6C
:1069700020625E4BBA00D358186A002803D01C224C
:10698000310004F0C1FD0C9B002B12D0574CBB0012
:106990001D596B6A002B03D1162004F0DDFD6862DF
:1069A000BB00E358586A002803D016220C9904F063
:1069B000ABFD0D9B002B11D04C4DBC006659B36A4A
:1069C000002B03D1142004F0C7FDB0622B59986A44
:1069D000002803D014220D9904F096FD380001F030
:1069E00089FD051E67D0414BBA00D358002B62D0F9
:1069F0001A6A3420002A00D11C389A6A002A01D071
:106A0000143080B20B9A002A01D01C3080B25B6A2D
:106A1000002B01D0163080B204F066FC041E4AD070
:106A20001822002104F088FC2620FFF76BFB019060
:106A3000002801D12B780193D0232370029B2000E2
:106A400063700A23294EA370039BBD00A371AB5949
:106A5000A780196A1830002905D01C22A06004F014
:106A600053FD200034307359996A002907D0030080
:106A700014221433E060029304F046FD02980B9B4D
:106A8000002B08D003001C221C330B9920610293B9
:106A900004F03AFD02987359596A002903D016226E
:106AA000606104F031FD6B462100187904F044FE6A
:106AB0003800FFF7E3FC05B0F0BD10220D9B0D99E7
:106AC0001B69A018236204F01FFD2CE70B9B002B11
:106AD00000D13FE7012D00D03CE7606A002801D0DB
:106AE00004F0E2FD1C210B982AE7C046C064FF1F9A
:106AF00010B5044C2068002803D004F0D5FD002315
:106B0000236010BDB464FF1F0B4B07B51A68002A41
:106B100001D100200EBD6946531C012012780731B7
:106B2000FFF772FC0028F4D002780123100018400F
:106B30001A42EED0EEE7C046D064FF1FF0B51F4FFB
:106B400001203B6887B0002B25D09B78059300F08F
:106B5000B3FB002821D00A20FFF7D4FA04000B2051
:106B6000FFF7D0FA164B05001E78731E9E413B6856
:106B7000F6B2191DD878FFF757FB3B682900DA7A7F
:106B8000043303929A79019302920090330020001B
:106B9000059A04F099FC07B0F0BDFFF7B5FF002897
:106BA00005D00620FFF7AEFA04000720D8E708203A
:106BB000FFF7A8FA04000920D2E7C046B464FF1F1B
:106BC000B064FF1F70B50A4E040033780D00FF2B30
:106BD0000DD0042004F088FB011E08D0D0230370E0
:106BE000CE3B45708370C470307804F0A5FD70BD55
:106BF0002843FF1F70B5040006200D0004F074FB4D
:106C0000011E0AD0D0230370CD3B8370054B447026
:106C10001B688580187804F08FFD002C01D0FFF7E9
:106C200067FF70BDB464FF1FF8B5264F06003B68D0
:106C30000D001124002B05D10522234B1B78134294
:106C400002D112242000F8BD204A10241268002A24
:106C5000F8D01278002AF5D0DB0719D52B789A1EC8
:106C6000012A1AD80C2004F077FC1324386000287D
:106C7000E8D000230A22437029000670023004F095
:106C800043FCFFF75BFF041E0AD0FFF731FFD9E793
:106C900000F012FB0028E1D1E4E7002BE2D0D0E7BE
:106CA0000B4B1B78032BCDD11D20FFF72BFA094B83
:106CB00018800028C6D0084B04211878074A04F031
:106CC000BBFCBFE7B464FF1FB164FF1FD064FF1FAC
:106CD000B064FF1FAE64FF1FDC64FF1F60EA0000AA
:106CE000F7B50193194B14001A78052306000F001D
:106CF00012201A4221D0012920D1154B1D68002DE8
:106D00001BD002201F2C18D8002C02D0019B002B76
:106D100013D0104B1F221E706E1C0021300004F097
:106D20000BFB01992200300004F0EEFB3100200043
:106D30002C70002F06D004F09FFBFEBD064B1220E6
:106D40001D68DCE704F088FCF7E7C046B164FF1F6C
:106D5000D064FF1F2843FF1FCC64FF1FF8B50F4E00
:106D600012243368002B17D01B780F3C834213D1B9
:106D700000250B4F0221387804F06EFB094B0421EB
:106D800038781D8004F068FB074B28001D803368AD
:106D90005C7004F061FA04002000F8BDB464FF1FC9
:106DA000DC64FF1FC864FF1FAE64FF1F70B50128BD
:106DB00023D11B4C2388002B03D01A4A1578002DB1
:106DC00007D0194B1B68002B02D01878FFF7C6FFBD
:106DD00070BD3B2B02D93C3B2380F9E7134E0221C7
:106DE000307804F039FBFA222388920002215A43BA
:106DF000307804F0B1FC2580EAE70B4B1B68002BD0
:106E0000E6D00B4B1B785B07E2D5084B02211878C4
:106E100004F022FB0022024B1A80FFF769FED7E73D
:106E2000C864FF1FAC64FF1FB464FF1FDC64FF1F56
:106E3000B164FF1FF8B51E4D2868002803D004F088
:106E400033FC00232B601B4E3068002803D004F075
:106E50002BFC00233360184F05243B78180020409A
:106E6000234221D0154800F02BFA3B78234213D05F
:106E7000202004F071FB2860002813D0202200217C
:106E800004F05AFA202004F067FB041E306005D09D
:106E90002022002104F050FA002004E0286804F0C9
:106EA00003FC2C601320F8BD00F00AFAF4E7C0469A
:106EB000D064FF1FCC64FF1FB164FF1F1C43FF1F82
:106EC00010B50A4C23681A1E0ED0002808D10130D4
:106ED000587004F0C1F9002805D02368002B02D0B7
:106EE0000021FFF787FE0122100010BDB464FF1FD0
:106EF000F7B5274E050033680191181E21D05C7844
:106F0000244F012C30D1FFF7FFFD002825D02000B1
:106F1000FFF7F8F80400412814D91F4B0221187814
:106F20001E4A04F089FB1E4B3C3C1C800222336845
:106F30005A703B78002B14D128000199FFF75AFEB4
:106F40000120FEBDFA2292004243002AEED0124BED
:106F50000221187804F000FCE8E7FFF7D3F80200FC
:106F6000F3E700233B70EBE73B78002BE8D10320ED
:106F700004F0BAF9011E08D0D0230370CC3B457051
:106F800083703368187804F0D7FBFFF7B1FDD7E7BB
:106F9000B464FF1FAC64FF1FDC64FF1F60EA0000E5
:106FA000C864FF1F10B51749838802008B4220D0A8
:106FB00011D815498B4217D0144900205B1899B29B
:106FC000012907D8926811785A425341D8B2FFF785
:106FD000F9FD012010BD0E4A00209B1807229BB22C
:106FE0009A424041C0B2F5E783681878FFF768FF1E
:106FF000F0E7836899785A78090218781143FFF707
:1070000077FFE7E70A20000006200000F8DFFFFF17
:10701000AFDFFFFF014B18707047C0462943FF1FC9
:1070200010B5064C207001F041FA207804F0ACF85D
:107030000521207800F062FD10BDC046DC64FF1F12
:107040000BB273B50D00002B00DBC4E0884B187841
:1070500004F0D2F9041E0ED00378912B0FD0A22B8E
:1070600000D1A1E0834B1878FF2852D0210004F012
:1070700063FB00284DD180200002684076BD437834
:107080000F2B76D013D8052B70D00E2BEAD1808829
:10709000794B98422BD8794B98421BD8784B984221
:1070A000E0D1A3681878591CFFF774F838E03E2B3C
:1070B000D8D18378032B74D06CD8012B6ED0022BDF
:1070C000D0D1704B1B68002B23D05B68002B20D0E5
:1070D00098471EE06C4BC0180C28C3D804F004FB82
:1070E0001DC2C2150BC20B0B0B3223C23C00674BF7
:1070F000C0180728B6D8664B1B68002B09D01B6840
:10710000002B06D0200098470AE0A3681878FFF704
:10711000C7F8200004F0D8F8ADE7A068FFF762F8E0
:1071200000289FD0F5E7A3681B78002BF1D0554BC2
:107130001B68002BEDD01B68002BEAD021005548BE
:107140009847EDE74F4B1B68002BE2D01B68002BE4
:10715000DFD021005048F3E7504B1B68002BD8D0FC
:107160005B68002BD5D021004348E9E7FFF7EAF937
:10717000CFE780884A4B984203D04A4B984200D0D0
:1071800070E7464B1B68002BC3D05B68002BC0D058
:107190002100D5E7153B012BBBD963E7FFF798FA30
:1071A000B7E7FFF77DFAB4E73F4B1B78042B07D115
:1071B00000236A4613800179408800F0C5FCA8E7E7
:1071C000364B1B68002BA4D05B68002BA1D00100BC
:1071D000364898479DE7012421420AD0294B1B6875
:1071E000002B04D05B68002B01D0002098470120C1
:1071F00043E78B070AD5264B1B68002B04D05B683E
:10720000002B01D020009847022036E704212800F7
:1072100008400D4200D131E7254E3388002B21D0A4
:10722000013B9BB23380002B1AD1FFF7DBF800281B
:107230000AD0204B1C70164B1B68002B04D05B68D7
:10724000002B01D020009847FFF7C6F8694601F0EF
:1072500001FD6846FEF7FEFF1D20FEF753FF30805C
:1072600004200AE7024B187804F0F6F8F8E7C04665
:10727000DC64FF1F2943FF1F0E20000001200000D7
:1072800009100000D464FF1FFEDFFFFFAFDFFFFF28
:10729000D864FF1F0C2000000B200000BC64FF1FFF
:1072A0000D20000013200000B164FF1FFFFF00004D
:1072B000AE64FF1FAC64FF1F10B501F09BF910BD59
:1072C000014B18607047C046D864FF1F0B88002030
:1072D000162B01D817230420014A13807047C0469B
:1072E0008664FF1F00207047074A0300118881420F
:1072F00007D091880020994202D1013080001018F7
:1073000070470020FAE7C046E464FF1FF0B58F78AD
:1073100006000D00C5B01E2F15D1FFF7E5FF051EB5
:1073200003D10024200045B0F0BD00223B00310015
:10733000C078009200F0B2FB0400A81C00F0D2FB61
:10734000FF23EB70EEE7264B062403931B78FF2BFD
:10735000E8D0182FE6D87B08224A013BDB000292D6
:107360009A589446002ADDD0029AD3185B68002B05
:10737000D8D00878002802D14B78012B02D10624FE
:10738000122FCFD107AFAB88697800976446AA68FF
:10739000A047041EC6D1AB78029A5B08013BDB0014
:1073A000D318390030005B689847041E0BD1AB78C6
:1073B000042BB6D0039A310010782200009700F019
:1073C0006DFB0400AEE76A78002AABD1AA7805A964
:1073D0003B88087130000A704B80FEF747FBA0E73E
:1073E0002C43FF1FE4B800111D4B37B50500984230
:1073F0000BD000290AD1FFF777FF002805D11948E3
:10740000FFF772FF002800D0058037BD01291AD18F
:10741000FFF76AFF041EF8D001235B420380A378C4
:10742000FF2BF2D0FE2B07D00023E078142200932C
:1074300029001E3300F032FBA01C00F053FB012397
:107440005B426380E1E70229DFD1013901F0BEF838
:107450000028DAD12800FFF747FF041EDFD1D4E768
:10746000FEFF0000FFFF0000022210B5074B524252
:107470001A80074801325A809A80DA8000F07EFA3A
:10748000044801F025F8002010BDC046E464FF1F49
:107490000D730011E97300110388F7B50400002B88
:1074A00002D102252800FEBD42680221137825483A
:1074B0005268FEF7A5FD00282ED0234F01253A88FB
:1074C000002AEFD0802321885B0201259B1A994274
:1074D000E8DC0C2004F040F8061E31D03B882288FE
:1074E0009C4600231800019561469DB2491989B256
:1074F000AA421BD8002801D062443A800023300001
:10750000082208C0210003F0FFFF104A1368002B77
:1075100013D100251660C5E76268022113780C4874
:107520005268FEF76DFD0028C7D1BAE760681D01FB
:107530004019418101330198D6E71A001B68E6E73C
:107540001325AFE752B900112A43FF1FE064FF1F64
:1075500050B90011014B18707047C0462C43FF1FF3
:1075600014230A0010B51A40194204D00122102138
:1075700001F048F810BD4B06F9D4012088434000C3
:10758000F8E710B514008B0604D50122102101F094
:1075900039F810BD08230A001A40194202D14BB233
:1075A000002B0FDA102101F02DF8002808D023005D
:1075B000F2331B78002BECD0F1342378012BE8D187
:1075C0000020E6E703208907FAD4E2E7F0B51F00C0
:1075D000184B85B01C68019002910392002C27D1B2
:1075E000200005B0F0BDA5683301ED186B89019A44
:1075F000934211D3029A93420ED8002F04D10A9BD2
:10760000002B10D12C00EBE73B002978039A686827
:10761000FEF7F6FC0028F2D10136B6B2A388B342D9
:10762000E1D82468DAE7A3680A9A5B891380E9E75E
:107630000026F3E7E064FF1F37B50C000A8849888D
:107640000123914217D3002A15D0651D23792A0002
:1076500002210A48FEF7D4FC102300280BD023791E
:107660006188208800242A000094FFF7AFFF0A23D6
:10767000A04200D0230018003EBDC04652B9001100
:1076800013B50A0008884988012388420BD80028CE
:1076900009D00024137905320094FFF797FF0A23DD
:1076A000A04200D02300180016BD13B50A000888B8
:1076B0004988012388420BD8002809D00024137977
:1076C00005320094FFF782FF0A23A04200D0230076
:1076D000180016BDF0B58BB003904A8808880E00DC
:1076E0000123824255D3002853D00023012704AC44
:1076F00023700022718813000092FFF767FF051EB8
:107700003ED02078002835D12B78022B18D1677015
:107710006A8983000130E31880005A806968022278
:10772000201803F0F1FE23780133DBB22370042B21
:1077300019D93B006889013080B2002BD9D01FE0F5
:1077400002236370122358436A89231804305A8035
:1077500069681022201803F0D7FE23780133DBB2CA
:107760002370002BE5D10C4A6B899B185A42534178
:10777000DBB2DFE76378012BE4D12B78022BC7D093
:1077800022780A23002A04D021000398FEF798F9F2
:10779000002318000BB0F0BD0100FFFF0F4BF0B548
:1077A00004001868002816D083685D89A54207D8B0
:1077B0008288AE18B44203DA12019A18934201D1BA
:1077C0000068EFE71E005F891036A74204D1002948
:1077D00000D00D801800F0BD3300EFE7E064FF1F1C
:1077E00070B505000C0008880021FFF7D7FF0300E3
:1077F0000120002B04D022002800197AFFF7C1FED7
:1078000070BDF7B50C00002501902300EE331B7806
:10781000AB4201D800200AE06B00E65A002130009C
:10782000E718FFF7BBFF002802D126800130FEBD1C
:10783000017A0198FFF794FE002802D03B8823804C
:10784000F5E70135EDB2E0E710B504000888002146
:10785000FFF7A4FF03000120002B03D02000197ABA
:10786000FFF77EFE10BD0000054B1B68002B01D109
:10787000180004E09A6852898242F6D198887047CD
:10788000E064FF1FF0B50E27002687B0039302AB1C
:10789000FF183E8005001F4B40891400984207D016
:1078A0002B78013000976A6880B2FFF78FFE0600E0
:1078B00002212B7818486A68FEF7A2FB00280FD037
:1078C0006C892000FFF7D0FF002802D0013C04198A
:1078D000A4B2039B002B00D01C80300007B0F0BD89
:1078E00002212B780D486A68FEF78AFB0028E7D151
:1078F00002212B780A486A68FEF782FB002807D02D
:10790000002EDED03B88A342DBD17489013CDFE747
:107910006C89DEE7FFFF000052B9001150B9001179
:107920004EB9001110B50C00FFF7DEFC0300022079
:10793000002B0AD0002C00D023609B781720FE2B50
:1079400003D00138FF2B00D1002010BD73B50D000E
:1079500001A904001600FFF7E5FF172805D0002E47
:1079600004D129002000FEF727F976BD012210215D
:10797000200000F047FE0028F3D0F6E7014B186026
:107980007047C046F064FF1F37B56B469D1D010070
:1079900004000222280003F0DFFB2B88B02B0ED15D
:1079A0002379122B09D12300FA331B78012B06D13E
:1079B0000121608800F0E0F801E01B2BF8D037BD12
:1079C00010B5054B0421187000F098F8FFF74CFD36
:1079D000FEF770FB10BDC046F464FF1F0020F0B539
:1079E0000BB20F0087B0834234DA274B187803F0CC
:1079F00003FD051E2BD00378A02B25D103AE31004B
:107A0000FEF7E4F8041E0BD1B378DB0724D51F4B37
:107A100006341B68002B03D03100688898470400A7
:107A2000A868002801D003F037FE002C08D1184ABE
:107A3000039B1340174A934206D0B3781B2B03D005
:107A40000121688800F098F8280003F03DFC8020B0
:107A50000002784007B0F0BD0F4B1B68002B10D020
:107A6000310068889847041EDAD07378002BD7D18C
:107A7000B27801A90A704B800C716888FDF7F6FF97
:107A8000CEE70624F1E7C046F464FF1FEC64FF1F55
:107A900000FFFF0000011200F064FF1FF7B5019026
:107AA000FC200D0017001E0003F01EFC0400132034
:107AB000002C12D0B02320002370089BF4226770A2
:107AC000658026710830002B08D0190003F01CFDDA
:107AD0002100019803F030FE0020FEBD089903F05C
:107AE0002BFCF5E710B5041E06D00078FD2803D85E
:107AF00003F062FCFF23237010BD00000A1F93B245
:107B000010B504000220032B05D882400020024B50
:107B1000D1529B189C7010BD1465FF1F0B8870B567
:107B2000043B04000D000220032B0BD80121200090
:107B300000F04CFD03001420002B03D0290020008E
:107B400000F0DEFB70BD000007B51300034A009291
:107B50000A00012100F02CFC0EBDC046857D0011FD
:107B600007B5019203220092024B0A00122100F095
:107B700049FC0EBD037E001107B56B4601AA1180BA
:107B80000449D88008780633012802D1190003F08F
:107B900023FD07BDF564FF1F0C4B10B518700023C3
:107BA000FF210B4A1380138193819380094A5380EC
:107BB0001370517293819372D174D382137551777C
:107BC00003F03AFC00F0FCF910BDC0462465FF1F2D
:107BD0001465FF1FF664FF1FF0B58DB06B460020E3
:107BE00003910C229B5E834200DBB0E05D4B187872
:107BF00003F002FC051E00D1A4E00378902B00D016
:107C00009DE006AF01004688380000F013FA79685D
:107C10000400002900D19CE03B88052B6ED13B89F4
:107C2000032B1CD905AC200000F0A2F86288172AAB
:107C300061D83989131D994231D17968237804318B
:107C40000291D90738D5607800F08EF9071E06D06A
:107C5000002303712378012B08D0132B23D0A868AD
:107C6000002800D178E003F017FD75E062880299E2
:107C700009A800F0A6F80290380000F08BF909AAD4
:107C80002378387A0192002231000092029A00F0A3
:107C900012F9380000F064F9029B002BDFD03000AD
:107CA00000F080F9DBE70378032BD8D162880299D2
:107CB00009A800F0D6F8DEE7122B13D1029909A823
:107CC00000F0B5F8021EEAD127498B88002BC6D0F8
:107CD000887909A92378019161780091310000F039
:107CE000EAF8BCE7002302AA93833000617809AA6E
:107CF000FFF72AFFB3E71D4B0993F6E7042B02D0E9
:107D00009A1F012AABD8184A043B9B00995A0029B4
:107D1000A5D0D218907831003A0000F0AEF80028D3
:107D20009DD13B88042B03D001213000FFF724FFB5
:107D3000012C04D1A868002801D003F0ADFC280074
:107D400003F0C2FA8020039B0002434018000DB0EC
:107D5000F0BD012800D182E701213000FFF70CFFC0
:107D6000EDE7C0462465FF1F1465FF1F01001700E3
:107D70000B7803704B784370CB788A781B021343DF
:107D8000438070470A88030002700A88120A427012
:107D90000A88012A06D14A8882704A88120AC2706B
:107DA0000420704702208242FBD14A8804309A7036
:107DB0004A88120ADA708A881A718A88120A5A71F5
:107DC000EFE710B50400012082420CD94B780A7805
:107DD0001B0213432380834206D1CB788A781B028F
:107DE00013436380002010BD022BFBD1CB788A782F
:107DF0001B02134363804B790A791B021343A38050
:107E0000F0E70B8803700B881B0A43704B88837064
:107E10004B881B0AC3708B8803718B881B0A4371C4
:107E2000CB888371CB881B0AC3710820704703007D
:107E30000120082A14D14A780878120202431A80D5
:107E4000CA788878120202435A804A790879120265
:107E500002439A80CA798879120202430020DA80AC
:107E6000704710B504000120022A05D100204B788C
:107E70000A781B021343238010BDF8B506001020BA
:107E80000F00150003F030FA04000120002C0ED082
:107E9000A0230C22290023806780201D002D07D0FD
:107EA00003F032FB2100300003F046FC0020F8BD57
:107EB00003F042FAF6E7F7B51E00009008AB142075
:107EC00017001D78019103F00FFA041E12D0A223AF
:107ED0000370019B47704380099B057146710C221A
:107EE0000830002B07D0190003F00EFB210000988A
:107EF00003F022FCF7BD099903F01EFAF6E737B547
:107F0000041E0FD04388002B0CD00025C1881323FA
:107F1000007A172201950095FFF7CDFFFF236580BA
:107F20006372257037BD000010B50C4904004A8803
:107F3000002A09D08B89002B05D00020CB8A022291
:107F4000834201D010BD012213000A2043430020C8
:107F50004032C854C81842800472F3E7F664FF1F29
:107F60000023438003707047094B00211A0010B5AD
:107F70005C88002C06D01C79844203D10A234B4331
:107F8000D01810BD01310A330329F1D10020F8E7E0
:107F9000F664FF1F10B50400407A03F00DFAFF23CA
:107FA000637210BD7047043010B580B203F01CFA44
:107FB000002803D00421494203F046F910BD000017
:107FC00070B50025104CA0682580A581A580A84229
:107FD00002D003F061FBA56000250C4C0C4B606DDA
:107FE0001D80230058331D70A84202D003F054FBBB
:107FF000656500256068002801D003F04DFB013560
:1080000008340A2DF6D170BDBC65FF1F6065FF1FE7
:10801000B065FF1F70B5041E09D1054D2880A881E9
:10802000A880A868002802D003F036FBAC6070BDC1
:10803000BC65FF1FF0B54B8885B0019300234360FA
:108040000A7905000F00022A00D07BE0CA88032AC3
:1080500017D98B685E7819783602DC78D8790E43A8
:1080600099781B7A24021B020C43034353495BBAE1
:108070000B80331D93421ED1042C04D0631F022BAE
:108080000ED9012015E0019A4D4B1201D35A002B55
:1080900006D00198FFF7BEFF4A4A13690133136106
:1080A0000421B8682E812C80494203F0CDF8686025
:1080B000002005B0F0BD434D042C06D0631F022BF9
:1080C0000FD9EB680133EB60DBE7019A3C4B1201FF
:1080D000D35A002B05D00198FFF79CFF2B69013381
:1080E0002B61374B30000293019B029A1B010193D5
:1080F000002301998C468B52130063449C800393A8
:108100009E81FFF750FF039B041E986016D0042148
:10811000B868494203F098F8FA880100043A200050
:1081200003F0F2F90199029AFB888A5A043B9B18E2
:10813000029A8B522B6801332B60A2E7AB690133A3
:10814000AB619EE71E4B0293019B1E01029BF35AFB
:10815000002B2DD002998C19A068002828D0012A64
:1081600026D1FA889B189BB27352A189994217D3E2
:108170009B1AC018B96803F0C7F9029BA289F35A89
:10818000934200D07DE700222B81A3882B80A36837
:108190006B60029BF2520B4A53680133536070E7E5
:1081A000084A9368013393600198FFF733FF68E74B
:1081B000044A536901335361F6E7C0462665FF1F41
:1081C000BC65FF1F2C65FF1F70B5051E15D10B4C3C
:1081D0000B4B1880230058331870606D002802D0B4
:1081E00003F05AFA6565250050356068002801D013
:1081F00003F052FA0834AC42F7D170BD6065FF1F3E
:10820000B065FF1FF0B51700A12285B09200019361
:108210004243394B06001B680C009B18D933FF33CF
:108220001D78FDF741FF0430854204DD3000FDF785
:108230003BFF0430C5B2BD4207D33A0000213000F5
:10824000019B03F011F805B0F0BD2900380003F0E0
:108250004BF92300C6B250331E700393019B2900D3
:108260006365380002F0E0FFCBB20293002B02D02E
:10827000039B01361E7000262300503303931B78A6
:10828000B34204D8606D002831D10020DBE7029AA8
:108290002800002A04D0013B1000B34200D028007F
:1082A000F700E719387003F0BFF9786000280ED0A6
:1082B0003A78019903F028F9019A3B780136D318EE
:1082C0000E4A0193D369F6B20133D361D4E7039B1D
:1082D00018706065A74205D1084A1320D36A01339C
:1082E000D362B0E7606803F0D7F90834F2E703F02F
:1082F000D3F900236365C8E73409FF1F2C65FF1F0E
:10830000F7B50D0007000421686802F09DFF2B8976
:10831000040003702B891B0A43702B8883702B8801
:108320001B0AC3702E8902250436F6B2F42E15D826
:108330001B4B9F4214D10C2002F0D6FF1135011EB9
:108340000CD0902303708E3B0371043B4380154B8C
:108350008460C680187803F0EFF900252800FEBD80
:108360005C237B43104AD3180093583301931B7846
:10837000002B0FD10300320038000099FFF742FFB5
:10838000019B05001B78002BE8D13800009903F011
:108390006BF8E3E7054A0725536A01335362DDE7CB
:1083A000FEFF00002465FF1F6065FF1F2C65FF1F97
:1083B000F0B587B0009017200F0016000193FFF76B
:1083C000F2FD1325041E19D00C98031E02D001994A
:1083D000201D9847030AE370052302AAA070043009
:1083E000908127700098667003A993800494FFF72A
:1083F00087FF051E02D0200003F04EF9280007B0C9
:10840000F0BD0000F0B587B01F000CAB1B780391E6
:10841000059301210DAB06001C78049200F0D6F8FC
:108420001425002821D02000FFF77EFD0135041E11
:108430001BD01149059B0A7803700132D2B2131E7A
:10844000C68001D101231A000B7022713000049BF9
:1084500003990097FFF7ACFF051E09D12300210007
:108460000648074A093302F0AFFF280007B0F0BD05
:10847000002363802370F8E72865FF1FFF7E00114B
:1084800030750000F8B505000E00064C064F236855
:10849000002B02D03100280098470434BC42F6D1AA
:1084A000F8BDC046CC65FF1FE065FF1F0123064AEB
:1084B0005B425380002313715362044A136053607C
:1084C0009360D36013617047E065FF1FCC65FF1FA9
:1084D0000200002310B506499C000859002801D16C
:1084E000625010BD0133052BF6D11320F9E7C046C9
:1084F000CC65FF1F034A5388181A43425841404233
:1085000010407047E065FF1FF0B585B002930AABDD
:108510001F780CAB1B88009008000E00019203939B
:10852000FFF7E8FF05001120002D1BD10E48FFF7D3
:10853000E1FF04001520002C14D006220B99A7712E
:10854000E01D02F0E1FF019B30002371029B290036
:108550006371009B66802370039B6562E381FFF774
:1085600091FF280005B0F0BDFFFF000010B5FFF738
:10857000C1FF04000220002C12D060880121FFF707
:1085800081FF606A002801D003F08EF828220021C4
:10859000200002F0D1FE012300205B4263802071A5
:1085A00010BD000030B5074A074C5588010013780C
:1085B0000020A54204D05B1A59424B41584210405A
:1085C00030BDC046E065FF1FFFFF0000084A10B540
:1085D00001230C00904208D0FFF78CFF031E04D04B
:1085E000037923405A1E9341DBB2180010BDC046E8
:1085F000FEFF0000024B1879431E9841C0B270473D
:10860000E065FF1F70B504000D001600FFF772FF54
:10861000002804D10D4B9C4200D0143070BD416A3B
:1086200003790520002907D012221A40102A02D10E
:108630000520002EF2D10F20DB06EFD5897E0C201D
:10864000A9428941494249420840E7E7FEFF00004C
:10865000030010B5002800D110BD0348034A41882B
:108660009142F9D09847F7E7E065FF1FFFFF000050
:10867000002330B5C45CCD5C6C40D4540133102B66
:10868000F8D130BD0F23002210B5C45C6400224332
:10869000CA54C25CD209013BF7D210BD02000100EE
:1086A00010B52032103102F09FFF10BDF0B58BB035
:1086B0000390102005931700049102F04DFF0090E5
:1086C000102002F049FF009B13240190002B05D0DD
:1086D00000280CD11324009802F0E6FF019B002B28
:1086E00002D0180002F0E0FF20000BB0F0BD102017
:1086F00002F032FF0600102002F02EFF13240500C6
:10870000002E00D1AEE0002819D01022002102F086
:1087100013FE32002900039802F066FF041E0ED1FA
:1087200033787F2B51D830000099FFF7ABFF009BC7
:108730001B787F2B53D801990098FFF7A3FF3000D7
:1087400002F0B2FF002D02D0280002F0ADFF002C95
:10875000C1D1102002F000FF0600102002F0FCFE44
:108760000290002E7CD0002878D03A000F322300EF
:108770000125121105D00F333B4015B25A42534127
:108780001BB26A1E1201002B33D0049BD2B2981880
:108790000099029AFFF76CFF013D10220021300082
:1087A00002F0CAFDADB2049F2D017D19AF4242D047
:1087B000002C33D0300002F077FF029B002B00D159
:1087C00089E7180002F070FF85E729003000FFF705
:1087D00059FF28002549009AFFF74AFFA7E729001B
:1087E0000098FFF74FFF28002049019AFFF740FF4C
:1087F000A5E70F210F4004998A18D9B28F4208D9F2
:10880000D15C06A819540133102BF6D1029A0199B4
:10881000C0E7791A48424141C901F2E73900300006
:1088200006AAFFF725FF3200039806A902F0DCFE36
:1088300010370400BAE7002CBCD13000029906AA18
:10884000FFF716FF320006A9039802F0CDFE0822BA
:1088500004003100059802F057FEABE71324A9E7A6
:108860001324AAE7002800D06EE733E758B90011B7
:10887000F0B58BB00F0016000225009000283FD005
:10888000002A3DD00B1DDBB21800029302F064FEFB
:108890001135041E34D0FDF747FD05003A0000995C
:1088A000201D02F009FEEBB20393E3702B0CDBB248
:1088B0002F0A00936370FFB22B0E2370A7700193F1
:1088C000FDF72CFD1022010006A802F0F5FD2100A5
:1088D000029A04AB06A8FFF7E9FE051E0DD1039B23
:1088E00008223370009B04A9B370019B7770F3706A
:1088F000301D02F0E1FDFDF71DFD200002F0D4FE69
:1089000028000BB0F0BDF0B58FB00D00149E0390A1
:1089100004920593002A03D1022420000FB0F0BD79
:10892000002EF9D00398FFF7E5FD1424071EF4D0BC
:108930007278337812021A43B3781B041343F27827
:1089400012061A43036A0192934201D30133E3D121
:10895000002D03D03B7901249B07DED5082200219E
:1089600006A802F0E9FC059B13240433DBB21800CF
:10897000029302F0F1FD051ECFD0059A0499043050
:1089800002F09AFD04223100280002F095FD390022
:10899000102210310AA802F08FFD2900029A06ABBE
:1089A0000AA8FFF783FE041E0FD1082206A908A813
:1089B00002F082FD0822311D08A802F02DFC0128DA
:1089C00007D101990398FDF7C9FC280002F06CFE5D
:1089D000A3E70124F9E7000070B51C4C05002368EB
:1089E000181E10D0002D14D11A78002A0CD1981C12
:1089F000083202F089FD02F06FFE0135002808D12F
:108A000023681D70012070BD0A331800082202F08F
:108A10007BFD2368002BF5D0122002F065FC061EBA
:108A20000DD0C1232168037045700231102202303D
:108A300002F06AFD23683100587802F07DFE20685C
:108A400002F032FE00232360DCE7C0460866FF1F09
:108A5000F8B504002020FDF755FB0D4EA700BB59CB
:108A60000500002B0DD000280BD0D878FF2809D1A5
:108A700008492A000C55F35907480333611802F0DE
:108A8000A3FCF8BD290002F08FFC0028F0D1F8E724
:108A90002466FF1F0C66FF1FA99C001170B5064DD0
:108AA00084006359002B05D0D87802F085FCFF22A2
:108AB0006359DA7070BDC0462466FF1F70B50600AA
:108AC0008CB00C00150000213022684602F034FC06
:108AD00031001022684602F0EFFC1D202100032225
:108AE000684402F0E9FC6846FFF7D8FD2D21040038
:108AF00003222800694402F0DFFC20000CB070BDA6
:108B0000F0B50700160097B001931CAB1D7830221A
:108B10001EAB00910AA800211C7802F00DFC102267
:108B200039000AA802F0C8FC1022002102A802F0B5
:108B300003FC0722310002A802F0BEFC072202ABB0
:108B40009818631E9C41019902F0B6FC02AB9C731D
:108B50002B005A1E934102AAD3730021102206A8AB
:108B600002F0EAFB06221D9907A802F0A5FC1A20D4
:108B700002ABC01806221F9902F09EFC1022009939
:108B80000EA802F099FC102202AB0EA908781C78FE
:108B9000013A6040D2B2087001330131002AF5D1A8
:108BA0000AA8FFF77BFD102212A904000EA802F00C
:108BB000ABFC102206AB0EA908781D78013A68407C
:108BC000D2B2087001330131002AF5D10AA8FFF7AB
:108BD00065FD044310222098E4B212A902F06CFC57
:108BE000200017B0F0BD70B50E0014008CB001006D
:108BF000102268461D0002F05FFC3100082204A824
:108C000002F05AFC2100082206A802F055FC684632
:108C1000FFF744FD04001022280008A902F04CFCD4
:108C200020000CB070BDF8B506000D000024371907
:108C3000AC4200D3F8BD02F09FFB030A3B70631CFB
:108C4000DBB201379D4203D90234F054E4B2EEE7BF
:108C50001C00EDE773B506000C000225002819D0B2
:108C6000002917D0032101A8FFF7DDFF6B469A7991
:108C70003F231A40013313436A463000937101A920
:108C80002200FFF71BFF051E04D10322E01C01A9EF
:108C900002F03AFC280076BD03785807DA08C00FC6
:108CA000D20080009B0710439B0F1843C0B270474F
:108CB00007230B40C908C9000B430370704700002D
:108CC00070B50400FFF7EAFE134DA4006359002BB2
:108CD00021D0186A002801D002F0E6FC2B59986ECA
:108CE000002801D002F0E0FC2B59D86E002801D0FA
:108CF00002F0DAFC2B59186F002801D002F0D4FCE6
:108D00002B59586F002801D002F0CEFC285902F0F0
:108D1000CBFC00232B5170BD2466FF1F0E4B80003F
:108D2000C35870B50C00002B0FD09D68002D0CD0DF
:108D30002B78201D0B706B784B70A97CFFF7B8FF68
:108D40002B7E23726B69E36070BD1022002120002E
:108D500002F0F2FAF8E7C0462466FF1F014B1860E4
:108D60007047C0462066FF1F074A030080008258F4
:108D700010B5002A06D0D088984203D1012901D12C
:108D8000FFF79EFF10BDC0462466FF1FF0B5264EBC
:108D900095B087000B93BB590500099112200A92E8
:108DA000002B31D0D888FFF7A5FB04001420002C3D
:108DB0002AD0280010A9FFF7B1FFBB591E781D6A01
:108DC000002E23D00895FDF7EFFA07000020FDF7ED
:108DD000F1FA0790A379E61D069310AD0CA9089847
:108DE00000F0E2FA0EA9280000F0D7FA0B9B0A99CE
:108DF0000493069B09980293079B0396019300979F
:108E00000EAB0CAAFFF77CFE15B0F0BDFDF7CCFA57
:108E100006903000FDF7CEFAE31DA779079310AB5B
:108E200006000893DAE7C0462466FF1F30B50C4CF5
:108E300085002A59030085B00120002A0ED01800B1
:108E40006946FFF76BFF2B591A78D888054B002A23
:108E500000D1054B6A46072100F0D9FB05B030BDB3
:108E60002466FF1F9B930011A993001130B5094C94
:108E70008500295985B010226846253102F044FB4F
:108E80002A591121044BD0886A4600F0C0FB05B076
:108E900030BDC0462466FF1F4594001130B5094C13
:108EA0008500295985B010226846353102F02CFB27
:108EB0002A591121044BD0886A4600F0A8FB05B05E
:108EC00030BDC0462466FF1F83940011F7B54D4F97
:108ED00086001020F4590D0002F03EFBF359206289
:108EE000186A132200286CD0033A29009C6802F00B
:108EF0000BFBF3591A780192002A58D11E6A227D81
:108F0000317B944651400122019F114201D16746B5
:108F10001740217D914339432175377B4F40BC4633
:108F200060460027800701D44F0817400121022026
:108F30008F40227D82433A432275377B5740BC469F
:108F400060460027400701D497080F400420227D87
:108F5000BF0082433A432275627D002794466046F3
:108F6000727B42400A4201D167460F400121627D77
:108F70008A433A436275777B5740BC466046002778
:108F8000800701D457080F400220627D7F00824392
:108F900017436775767B00227E40760701D4BA08B6
:108FA0000A400426617D9200B1430A4362756A78E3
:108FB000002A08D06278002A05D005220533DA7726
:108FC00000221000FEBD04222979114205D1A17CA6
:108FD000114202D10533033AF1E7019A21782C7846
:108FE000002A02D10A002100140018220429E8D81E
:108FF000042CE6D805206043034A05331218525C5E
:10900000DDE7C0462466FF1F68B9001110B50A00ED
:109010001121024B00F0FBFA10BDC046DF94001195
:109020000B0030B587B001AD2B806B4604001100FA
:10903000981D082202F068FA2A000B212000024B3A
:1090400000F0E5FA07B030BD0795001110B50A0031
:109050001121024B00F0DBFA10BDC0465B950011F8
:1090600013B50B0011006A4613706B46040006220C
:10907000581C02F049FA6A4608212000014B00F012
:10908000C6FA13BD7B95001110B50A001121024BE1
:1090900000F0BDFA10BDC046CB9500117FB50500AC
:1090A0000B4BAA00D4580800002C0FD0666F237F0A
:1090B000E28821780396266F0296E66E0196A46EEA
:1090C0000094FDF709FC2800FFF7FAFD7FBDC046BC
:1090D0002466FF1F10B51721FFF7E0FF10BD000049
:1090E00070B50A000D00064B0221040000F08FFA53
:1090F000060029782000FFF7D1FF300070BDC04680
:10910000AB94001170B586B000236A461370836873
:1091100004001D78681E0A2859D801A902F074FAC3
:10912000060633373B3F43474B4F5300180000F0D0
:1091300042F9062312284BD000281BD16088FFF784
:10914000D9F90823002813D04279002A47D1264BA9
:109150001A78072312070BD5244B1A680723002A15
:1091600006D01668002E03D0290001AAB0470300DC
:109170006A4613706B461B786088002B2AD1FFF774
:1091800067FC06B070BD180000F06CF9D4E7180059
:1091900000F087F9D0E7180000F093F9CCE7180049
:1091A00000F0ADF9C8E7180000F0C3F9C4E71800F3
:1091B00000F0F6F9C0E7180000F0F6F9BCE7180077
:1091C00000F013FAB8E7180000F013FAB4E7072329
:1091D0006A46137069466088FFF782FFD1E705236E
:1091E000012AC5D1024BB8E7B164FF1F1C66FF1FFF
:1091F0002066FF1FF8B52C4F8600F35904000D00C0
:10920000002B40D0DA8882423DD15A78062A33D1E9
:109210001A78002A2ED0012099681A6A097D014225
:1092200006D0157B054203D007225A700120F8BDF5
:109230000220014204D0157B054201D00922F4E747
:109240000420014204D0127B024201D00B22ECE741
:10925000164B1B68002BE9D05B68002BE6D0200082
:109260009847BB5900215B78122BDFD12000FFF714
:1092700015FFDBE70E4BECE7112A04D1002900D0E3
:1092800032252900F2E7002D08D12000FFF732F93E
:10929000002803D010230279134303712100280012
:1092A000FDF798FAC2E7C0462466FF1F1C66FF1F41
:1092B0002066FF1F70B50E4E8500AB590400002BD1
:1092C00013D01B78002B11D10A4B1B68002B04D044
:1092D0005B68002B01D02000984773595B78122BF4
:1092E00003D100212000FFF7D9FE70BD024BECE74F
:1092F0002466FF1F2066FF1F1C66FF1F094B8000AE
:10930000C3581020002B0CD01A6A002A09D09B6881
:10931000002B06D0127A1B7E101C9A4200D9181C12
:10932000C0B270472466FF1F70B503000D00140023
:109330000220002A30D000292ED013700B78081D8F
:1093400053704B789370FFF7A7FCE0700120022167
:109350002B7A23716B7B034063716A7B0A40134352
:10936000042263716E7B1640334363716E7BF60893
:10937000F600334363712B7B0340A371287B0140CC
:1093800000200B43A371297B0A401343A3712A7B5E
:10939000D208D2001343A37170BD10B50A000100BA
:1093A0000120FFF7C1FF10BD10B50A000100022027
:1093B000FFF7BAFF10BD70B506000C000220002EAA
:1093C00030D000292ED07378201D0B70B3784B70ED
:1093D000F178FFF76DFC01223579257271794B1018
:1093E0000800134093401040034388101040800051
:1093F000C9080343C9000B436373B1794B100800DC
:109400001340934010400343881002409200C90863
:109410001343C9000B4321202373FCF773FE8542DD
:1094200001D2122070BD2220257AFCF76BFE854206
:10943000F7D823781820042BF4D86378012BF1D8BF
:109440000020EFE7030010B50220002909D0002B0F
:1094500007D00322481C0A7019000D3202F054F89C
:10946000002010BD03000222080010B5002B06D01A
:10947000002904D00E32591C02F046F800221000D8
:1094800010BD030010B50220002909D0002B07D021
:109490000422481C0A7019000C3202F035F8002032
:1094A00010BD10B5FFF7DEFF10BD0300022000293C
:1094B00006D0002B04D0052200200A701B784B70C8
:1094C000704703000220002B08D0002906D05B78EB
:1094D00000200B70013B082B00D9183070470300A7
:1094E00010B50220002909D0002B07D00622481C05
:1094F0000A7019000A3202F007F8002010BD10B5FA
:10950000FFF7B0FF10BD02000B00022010B50029CC
:109510000ED0002A0CD007211970118859701188BB
:10952000090A997011180822D81C01F0EDFF0020DB
:1095300010BD03000A00022010B5002B0CD000293A
:109540000AD099785878090201431180901CD91CDF
:10955000082201F0D9FF002010BD030010B5022041
:10956000002909D0002B07D00822481C0A701900D6
:10957000921801F0C9FF002010BD02000B0002206C
:1095800010B500290BD0002A09D0092119701178D3
:1095900018185970511C062201F0B6FF002010BDAA
:1095A00010B5FFF75FFF10BD02000B00022010B5E1
:1095B000002A09D0002907D0517819701118062205
:1095C000581C01F0A1FF002010BD030010B50220BF
:1095D000002909D0002B07D00A22481C0A70190064
:1095E000063201F091FF002010BD10B5FFF73AFFE1
:1095F00010BD02000B00022010B5002A06D0002981
:1096000004D018005178FFF753FB002010BDF0B5CF
:1096100085B017001E006A460623050008009181E8
:109620009380FEF7C0FC1324011E02900CD038007A
:10963000B047041E05D1280001A9FEF76FFA041EE9
:1096400002D0029802F028F82800FFF701FA200063
:1096500005B0F0BDF0B504008BB0019115000021FC
:10966000102202A801F068FE334EA700B859002866
:109670003CD0C388A34239D10378002B36D142783D
:10968000062A18D102000100553235310C3006ABE4
:10969000FFF7A9FA002829D12000FFF72FFE0200CA
:1096A00006A902A801F030FF200002A901F0B4FFD2
:1096B00001200BB0F0BD816E002917D00B8A112A52
:1096C00028D19D420ED101981231093A01F0A4FD32
:1096D000012807D1BB5920009D6EFFF70FFE29001E
:1096E0000200DEE732212000FFF7D8FC2000FEF761
:1096F00001FF061E1BD0416A002918D00B8AAB421D
:1097000015D108220198123101F086FD01280ED1F1
:10971000716A0AE09D42E9D108220198123101F0F4
:109720007BFD0128E2D1BB59996E8A7EB9E7200002
:1097300001F0FAFDBCE7C0462466FF1FF0B56B4D93
:1097400087007E5985B0337802900393002B00D0B8
:1097500087E0B368346A01937078062817D1012234
:109760001B7D134202D0217B114218D102221342E9
:1097700002D0217B114251D10422134203D0237B1A
:10978000134200D08BE0019B5A7DEB5991E00738E2
:109790000428F8D801F038FF032E42678300B36E27
:1097A000002B03D11C2001F0D7FEB066EB599C6E54
:1097B000002C1CD010220021200001F0BDFD0298D9
:1097C000FFF79CFD01002000FFF72DFA01F0D4FD0A
:1097D0002082200008211230FFF725FA0298FFF7B7
:1097E0008DFDA076EB592100D888FFF70FFC0822E9
:1097F000EB591CE0B36E002B05D01A00198AF088D3
:109800001232FFF70DFC0222019B197DEB59114228
:109810003DD0207B10423AD0073208E0F488FCF7B4
:10982000DBFD01002000FFF711FC0A22EB595A7002
:10983000029B9C002A595378073B042B11D8D088EF
:10984000FEF758FE00284ED0C3895A08D21828497E
:10985000029B0298CB542B5941180433254801F040
:10986000B3FD05B0F0BDFCF79FFD0300012083426E
:1098700001D100200393EB59DE88FCF79BFD03998F
:1098800002003000FFF7ECFB019AEB59117D042236
:1098900011420CD0217B114209D00B22C7E7F68878
:1098A000FCF73CFD01003000FFF7EEFB6BE7019A8F
:1098B000527D01210A4204D0607B084201D00C2273
:1098C000B5E702210A4204D0607B084201D00E2293
:1098D000ADE704210A4204D0627B0A4201D0102283
:1098E000A5E71222A3E7FA225200B0E72466FF1F81
:1098F0002866FF1FB39C001110B5064B1A7804238D
:10990000100018401A4200D00348FFF727FA002041
:1099100010BDC046B164FF1F3043FF1F70B5040087
:10992000FFF7D4FA051E43D12000FFF77FFA234E3C
:10993000A400A0598268937CDB0708D50321036A41
:109940001B790B40012B02D1017F0B430377431D91
:10995000D97F8B1E022B0DD8022900D00121C0888F
:10996000FCF790FF042133591A7F59700A431A7784
:10997000280070BD01290CD1022310224370002160
:109980000C3001F0D9FC305910213530FFF74BF97C
:10999000EEE70529ECD10223D118437010220C30D8
:1099A00001F0B2FD04233259117F0B431377EAE72C
:1099B00008251828DCD1053DDAE7C0462466FF1FDC
:1099C000F0B58BB0059143887E4F9E00F459150089
:1099D0000493002C15D1012902D000200BB0F0BD5A
:1099E000101D57781678FFF757F9EB68320002938D
:1099F0002B7A0499019300903B002000FCF70CFFA8
:109A0000EBE7E388049A934201D00820E6E7237845
:109A1000012B00D1D4E0059B581E092800D9CFE0C6
:109A200001F0F2FD05CE0A29CC506C859AB22900CE
:109A30000498FFF773FFD1E720002900102245307A
:109A400001F062FDB9594B78042B02D1013B4B70F8
:109A5000C3E70B000A00253335320C310498FFF7B9
:109A600095F90498FFF702FA0522431E9841BB5965
:109A7000C0005A70B2E7200029001022553001F0D2
:109A800043FD049B4F4C9D00295904980A0006ABE6
:109A900055320C31FFF77AF929591022453106A8C1
:109AA00001F0BAFB012808D10498FFF7F7F90590F7
:109AB000002804D106222B595A7005988EE70823F6
:109AC0000593FAE763780C2B7AD1E36E002B03D170
:109AD0001C2001F041FDE066BB59D86E00286FD014
:109AE0001022290001F010FDBB590498DC6EFFF72D
:109AF00005FC0D22A076BB595A706EE7E06E002877
:109B00005ED063780D2B5BD12B8808220382A91CC1
:109B1000123001F0F9FCBB599A68517D02221142C2
:109B200026D0186A407B104222D00C32E4E76378DA
:109B30000E2B45D1236F002B03D1162001F00CFD15
:109B40002067BB59186F002803D01022290001F0AC
:109B5000DBFC0F22BB59CFE763780F2B30D1206F8E
:109B60000622691C103001F0CFFCBB599A68517D68
:109B70000422114203D0196A497B1142D5D1002138
:109B80000498FFF78BFA28E7636F002B0DD0BB59C1
:109B9000586F0028F3D01022290001F0B5FC0122F3
:109BA000BB5952425B6F1A61E9E7142001F0D4FC03
:109BB000BB5960675B6F002BE9D126E72978DFE7A7
:109BC00007200BE72466FF1F10B5064C207001F03C
:109BD00073FB06212078FDF791FF0348FEF778FC20
:109BE00010BDC0463766FF1F698D001100200BB203
:109BF00070B50D00834216DA264B187801F0FCFB95
:109C0000041E0DD00378922B0ED0A02B37D0224B00
:109C10001878FF283AD0210001F08EFD002835D1B8
:109C200080200002684070BD43780E2B0BD03E2B85
:109C3000EDD18378052B12D0082BE8D1817980886B
:109C4000FFF7D8FA08E0154B82889A42DFD1836883
:109C50001878591CFEF7C0FE002817D1D7E7104B23
:109C60001B785B0712D50F4B1B68002B0ED09B682F
:109C7000002B0BD0C289811D80889847ECE7FFF745
:109C800041FAA068002801D001F006FD200001F093
:109C90001BFBC5E73766FF1F2943FF1F1820000085
:109CA000B164FF1F2066FF1F10B50078FFF712FA9E
:109CB00010BD10B50078FFF7FDFA10BD0C2343432B
:109CC000084A10B59B185A68002A03D0012901D10F
:109CD000904710BD9B68002BFBD00029F9D1984715
:109CE000F7E7C0465466FF1F01238340094A10B5B9
:109CF000946B1C439463506B98435063D46B200067
:109D00009843012901D120001843D063116B0B4304
:109D1000136310BD00800040F0B500240127154BEF
:109D200085B0DA6B144E03921A6C0192DA64019BCF
:109D3000E3403B4217D0039DE5403D400295E5B22C
:109D400002992800FFF7BAFF316A736A002908D028
:109D50003900002B01D0029979402800FFF7C4FF99
:109D600001E0002BF9D101340C36172CDFD105B0FE
:109D7000F0BDC046008000403866FF1F064B012141
:109D80005A68C2400A4204D01B68C3401800084009
:109D900070471B6DF9E7C0460080004030B50324D2
:109DA00044430F4BE25C1B199C785D7801232D1B0B
:109DB0000135AB40013BA340A140DB430C0012281E
:109DC00007D80849920052181168194021431160C0
:109DD00030BD054A11680B4023431360F8E7C046C5
:109DE000AFB9001108F0004014F00040C21F70B578
:109DF000D4B20623092C0BD80125084C9540002924
:109E000008D00021FFF7CAFF23682B4323600023FB
:109E1000180070BD2368AB43F8E7C0460038004027
:109E2000214BF0B51B185B78022B21D1032444434E
:109E30001E4A1F4EA35C121994780122150085401A
:109E4000B76B013CE4B23D43A240B563194C122804
:109E500015D89B0000290CD117495B1899680A4353
:109E60009A600123205C154A834011680B431360FC
:109E7000F0BD11495B18996891439960F1E70E4B69
:109E800000290DD159690A435A61225C1328E8D090
:109E90000123203A93400A49086803430B60E7E72F
:109EA000596991435961F0E73866FF1FAFB9001156
:109EB00000800040F4B9001100F00040A0F0004024
:109EC000A4F00040F8B500241B4E1C4D1C4B1B5D3C
:109ED000012B1FD1194A9269E2401A420BD001228C
:109EE000B25693402200143AD2B2022A09D8154938
:109EF0004A6913434B61013402360C35172CE5D106
:109F0000F8BD0022B2560F499200521891680B43D7
:109F10009360F0E7022BEED1E7B23800FFF72EFF97
:109F200001235840C1B23800FFF77AFF3800FFF72D
:109F300025FF6877DFE7C04681B900113866FF1F4B
:109F40003966FF1F00F00040012202388240054BB5
:109F5000002903D059690A435A61704759699143EE
:109F60005961FAE700380040F8B50E0001210F00F2
:109F70008740114A0400D368FD43BB43D360831E6E
:109F80008B4201D8FFF7E0FF00212000FFF72EFFF2
:109F90000A4A0B4B5168012E05D139431B195160F8
:109FA0005E700020F8BD2940516002221C196270C9
:109FB0009A6915409D61F4E7003800400080004038
:109FC0003866FF1F012210B58240074B002906D0DA
:109FD00019680A431A600121FFF7C6FF10BD19680E
:109FE00091431960F7E7C046008000400C2370B52C
:109FF000002543430A4A29009B181D70094B0400A1
:10A000001B185D70FFF7B0FF0123A340064928002D
:10A010000A681A430A6005490A689A430A6070BDD3
:10A020005466FF1F3866FF1F3480004030800040B8
:10A03000F8B50C244443134B0500E4186368002B67
:10A0400003D1A3681220002B1AD0022201270E4B45
:10A0500000215B195A7028002770FFF785FF63689D
:10A060001E1E08D0A3683E00002B04D02800FFF776
:10A0700085FE4640F6B228003100FFF735FE00208D
:10A08000F8BDC0465466FF1F3866FF1FF7B5C420F1
:10A09000FF222B4B80001958002491433F3A0A437A
:10A0A0001A508022274F5202274E1A60274B1D5DFF
:10A0B000002D21D0A31E012B03D80121E0B2FFF710
:10A0C00043FF012D18D11F4B9B69E3402B4213D056
:10A0D000E3B218000193FFF751FE01000198FFF76A
:10A0E00071FFE3B2143B022B1DD801217156184AAF
:10A0F0008D405369AB4353613B7F002B0DD0E5B2DC
:10A100002800FFF795FF2800FFF738FE7B7F01004E
:10A11000834202D02800FFF7D1FD01340C3702360C
:10A12000172CC3D1F7BD012100237156F3568D4082
:10A13000074A9B009B189A68AA439A60DCE7C046CE
:10A1400000E100E03866FF1F81B900113966FF1F8A
:10A1500000F0004010B501210400FFF705FF0123C6
:10A16000044A002011194B70A34091690B4393617D
:10A1700010BDC0463866FF1F70B50E001500040004
:10A18000FFF734FF0C236343094A20009B189D60AE
:10A190005E60FFF74DFFF021064B074A8900051E60
:10A1A0005A5002D02000FFF721FF280070BDC046A2
:10A1B0005466FF1F0000FF1F199D001170B5134D5D
:10A1C00007202C78002C1FD1982221005200280053
:10A1D00001F012FA0123C420FF222B700C4B8000E7
:10A1E0001C635C630B4B1C605C600B4B1958914308
:10A1F0003F3A0A431A50802252021A600D20074A41
:10A20000074901F031FA200070BDC0463866FF1FD3
:10A2100000800040A0F0004000E100E08DA00011AF
:10A22000C59E0011030010B50620072B09D8054A6A
:10A23000137001F079FAD7210020034B034A8900FB
:10A240005A5010BD5843FF1F0000FF1F8D1BFF1FFA
:10A2500070B51D0002240C2910D8094ACA40D20743
:10A260000CD5FBF75BFF041E08D1059A0499280062
:10A27000FBF770FFFCF7DEFDFFF73EFB200070BD33
:10A280001210000030B50D7802232C009C431842B8
:10A2900001D02B431C0008252300AB43284201D0EA
:10A2A0002B00234320241D00A543204201D01C4342
:10A2B00025002A230D70184204D011781E3B0B4351
:10A2C000137030BD0028FCD10C2113788B43F7E7C5
:10A2D000F8B51D0006AB1B88140007AA0E000B2062
:10A2E0001778002B27D10A78022A49D14A6850787A
:10A2F00011780002244A08438018042840D801F04D
:10A3000083F903121D1B2300F06801F00DF9021CF4
:10A31000C0B2B84200D93A1CD2B22000F1682A80FB
:10A3200001F0F2F806E00222F3681B882A8023700D
:10A330001B0A63700020F8BD0622EEE701232B8084
:10A34000F3681B782370F5E7F368002B16D008221A
:10A350002A801A8822701A88120A62705A88A2709B
:10A360005A88120AE2709A8822719A88120A6271D7
:10A37000DA88A271DB881B0AE371DBE72B80D9E75F
:10A3800001202B80D7E7C04600D6FFFFF7B51600A7
:10A390000A781D0008AB1F880C000123022A18D17F
:10A3A0004A685078117800022B4A08438018032825
:10A3B0000FD801F029F902254439E06801F0B4F81A
:10A3C000C0B20723B84204D37B190193152B02DDD9
:10A3D0000D231800FEBDE0682A003100C01901F00D
:10A3E00093F86B4600209B88E268D0541B4B1B6897
:10A3F000834203D01B68834200D098470023E8E7DC
:10A400000B23002FE5D1022DE2D1737832781B02A5
:10A410001343E2681380114B1B68002BEED01B68BE
:10A42000002BEBD00120E8E70B23002FD1D1062D24
:10A43000CED12A003100E06801F066F8DEE70B2398
:10A44000002FC6D1012DC3D132787533012AC0D86F
:10A45000E3681A70D2E7C04600D6FFFF4468FF1FCA
:10A4600070B50C001500072837D801F0CDF804149A
:10A4700036361B36242E182015290BD8184E1622D6
:10A480000021300000F058FF22002900300001F0C8
:10A490003BF8002070BD18200229FBD11288114B17
:10A4A0001A80F6E718200829F4D10A000E4829007E
:10A4B00000F052FEEDE718200129EBD10B4B10788C
:10A4C0000B49DA69FFF7DEFEE3E718200129E1D145
:10A4D000064B10780749DA6BF4E70220DAE7C0464A
:10A4E0002C68FF1FD643FF1FCC43FF1F5C43FF1F99
:10A4F0008443FF1FA443FF1F030010B50020DB07A8
:10A5000004D50721024A034800F08CF810BDC0466C
:10A510000CBA00115C43FF1F054A030010680028B5
:10A5200003D082889A4201D1806870470068F6E7BC
:10A530003C6AFF1F0A88030008009A4204D08A88F8
:10A5400004309A4200D0002070470000F8B5F22293
:10A5500000230D4F0D4E7968050042433370994238
:10A5600000D07B600A4C0021200000F0E5FE0023B3
:10A570001A007C60AB4202D100203370F8BD013379
:10A580002280DBB2F234F5E7346BFF1F326BFF1F22
:10A59000406AFF1F73B56B460190060068461500C0
:10A5A0001980FCF779FF041E11D1002D0FD0768998
:10A5B000002E11D00C2000F0CFFF00280ED0084A4A
:10A5C0000460136886808560002B02D11060200033
:10A5D00076BD1A001B68F7E70224F8E71324F6E7B4
:10A5E0003C6AFF1F012100220A4B10B549420A4C68
:10A5F000198099809A719A70084B207001201980F7
:10A600005A60FFF7A3FF2078FCF7A4FF0448FDF78A
:10A610005FFF10BD4C68FF1F3C6BFF1F346BFF1FBB
:10A62000D1A60011022310B5002802D0FFF7B2FF17
:10A630000300180010BD0000030010B50020DB0768
:10A6400004D50421024A0348FFF7A4FF10BDC04609
:10A6500020BA0011DC43FF1FF0B50E2687B003932C
:10A660000CAB1F8802ABF6180500080031000292FF
:10A67000FDF794F804000120002C0FD03088FFF77C
:10A680004BFF03000E20002B08D05E68002E05D083
:10A6900021002800039B029A0097B04707B0F0BD45
:10A6A0000A4B10B5984207D10122002352420A807A
:10A6B0008B708A808B7110BDFFF73CFF0028FAD0A9
:10A6C00001235B42038000238370F4E7FFFF000057
:10A6D000F8B5050001290AD1134E00243388F2276A
:10A6E000AB4219D028001149FFF7DAFF06E0022932
:10A6F00004D10139FDF76AFF0028EDD0F8BD3B0019
:10A7000063437268D018D35A002B09D03A00002155
:10A7100000F012FE0134E4B2054B1B78A342EED8E0
:10A7200001235B423380DDE7346BFF1F4C68FF1F62
:10A73000326BFF1F10B5FFF7FDFE030000208342C0
:10A7400000D0987810BD0000F0B589B01C000EABA9
:10A7500080CB03901E8810AB1B78049202930B7A77
:10A760000D00DB0616D42B780593022B24D0049819
:10A77000FFF7D2FE002812D003689C46002B0ED0B3
:10A78000029B2200019329003B0064460398009637
:10A79000A04705E00498FFF7BFFE002802D10E2075
:10A7A00009B0F0BD8368002BF9D00A222900039874
:10A7B00098470028D7D0F3E76B6858781A786B4B26
:10A7C000000210439842D2D8043B984210D2684B02
:10A7D000984242D015D8674BC0180128C7D80B2023
:10A7E000002EDDD1EB681A7859683A80200028E005
:10A7F000614BC018032800D979E000F005FF846A96
:10A80000789E5E4B9842B2D10B20002EC8D1012316
:10A810003B80EB6831001B7823706889013080B27F
:10A82000FCF7BCFF3A88031E0ED0017802328A186A
:10A830003A80428962704289120AA270596802788D
:10A84000E01C00F061FE06E004323A803100042290
:10A85000601C00F071FD0020A2E70B20002E9FD1AC
:10A86000EB6807A91E8804233B80330A300026705A
:10A870006370FCF793FF051E28D004AB9A890E2362
:10A8800004A95B183E49C668FCF7FCFF00280BD101
:10A890002B783C486A680599FBF7B2FB002803D186
:10A8A000012304AA5B42D3813278022A06D171685F
:10A8B000201D00F029FE3B8802333B800E2304AAB2
:10A8C0009B181B88A3701B0AE370C4E704ABDE81EE
:10A8D000F4E70B20002E00D062E7E9680398FFF749
:10A8E00029FF02233B802070000A6070B3E70B2031
:10A8F000002E00D054E70222EB681B883A802370B8
:10A900001B0A6370A7E7E86800F00EFEC2B20300FE
:10A910000720B24200D243E70DD00299DBB2711892
:10A92000994202DB921BD3B20293029BE9681A00A0
:10A930003B8089195AE70023F6E70B20002E00D050
:10A940002EE70722EB683A801A7822705A786270F4
:10A950005A88A2705A88120AE2701A792271DA882B
:10A960006271DB881B0AA37175E7C04604290000E9
:10A970000228000000D8FFFFFFD6FFFF03280000D9
:10A98000FFFF000050B90011F0B58DB06B460020FC
:10A99000089120229B5E83423DDAA64B187800F096
:10A9A0002BFD071E32D00378B02B2CD10079023852
:10A9B00016281FD800F080FE17001E001E001E0083
:10A9C00031001E0096001E001D011E0052011E00D7
:10A9D00073011E00CD011E0050021E001E001E004D
:10A9E0008E021E00E302944B94491B8878880B80EA
:10A9F000FBF746F83800FCF7C7FF914B1B68002BAC
:10AA000001D038009847380000F05EFC8020089B99
:10AA10000002434018000DB0F0BDEE22002187482F
:10AA200000F08AFC0BAA3B7B7989388900923A00B6
:10AA30000D32FCF7CBFD0400804B1B78002C3FD17E
:10AA400046E0804B788805937F4B4100CB5A0BAE94
:10AA5000073BDBB232880293002301937B4B21003A
:10AA600006930093059BFFF76FFE744D002810D1ED
:10AA7000069B3A8A1B889A420BD1380005991230FE
:10AA800000F0CAFB002804D02B7862899B00EB18E9
:10AA90005A80162306A81B18328820007989FCF7F3
:10AAA000F1FE2B7804009A00AA1851880029C3D01F
:10AAB0000133DBB22B70002807D006A9C98A918028
:10AAC000634A12889A42BCD802E00121494291802F
:10AAD000002B04D059497888FBF706F88AE73E89AD
:10AAE0000A2479E000253E89574B06937B88069A15
:10AAF0005B009B5A033B9D4202DB002DF0D05BE0E4
:10AB0000162206A812183B7B798900923A00300081
:10AB10000D32FCF75BFD0590002858D04689017A7C
:10AB20007888FCF71DFD041E44D1464B78880793B6
:10AB3000069B4100C95A454B0439C9B206AAD28ABC
:10AB400006930291019400930599079BFFF7FCFD82
:10AB5000041E2FD1069B39491A88931C002D26D13B
:10AB60004B807988384B4900CB5A5119033B8B42B3
:10AB700020DD059B31485B8941190B71A91C01350A
:10AB8000C9B2EDB2059145191B0A2B71059B2D49E0
:10AB90000433181800F0B8FC2C4B059A1B88D31806
:10ABA000DDB22C4B9E4205D00136B6B29CE74988F7
:10ABB0009942D6D0002D0CD0204C2800618800F09E
:10ABC000ABFC207021007888FAF79EFF12E7059C05
:10ABD000F0E7002C00D183E77B78142B00D109E744
:10ABE00016493B794E800B700C717888FAF73EFF5E
:10ABF00000E7162406ABE41821003889FCF7CEFDE7
:10AC0000011E00D1B7E1788822880F4C45002C5BEB
:10AC10000A4D013CE4B2029400240F4B01940095CC
:10AC2000FFF792FD041E00D014E129007888FAF79E
:10AC30007BFFDFE63C6BFF1FC842FF1F5468FF1F0E
:10AC40004868FF1F4869FF1F8464FF1F386AFF1FA1
:10AC5000C642FF1FFFFF00005668FF1F162406AB09
:10AC6000E41821003889FCF799FD011E00D182E12A
:10AC700078882288AE4C45002C5BAE4D013CE4B296
:10AC800002947C89AC4B01940095FFF75DFD041E96
:10AC900000D0DFE029007888FAF750FFAAE6002507
:10ACA000A44B1D803B00F6331B78A24A788807929C
:10ACB000AB4208D99E4B12880693069943005B5A13
:10ACC000013B9A4203DB0799FAF742FF92E616240A
:10ACD0006B00FB18059306ABE418059B210018894F
:10ACE000FCF75CFD011E03D1059B01241E8973E75F
:10ACF0007888924B2288069C099343001B5B904EF8
:10AD0000013BDBB20293002300960193099BFFF7FE
:10AD10001BFD041E02D0059B1E895DE77B88069AF9
:10AD20005B009B5A079A108832881218934202DC03
:10AD30001B1A013B33807F4C02303288099900197D
:10AD400000F0E2FB2388328801359B182380EDB2A6
:10AD5000A8E70BAA3B7B7989388900923A000D322B
:10AD6000FCF734FC00250590059B002B04D10A2438
:10AD7000002D00D16EE060E0059B7888197AFCF721
:10AD8000EFFB0100041E63D1694C6C4B788806947C
:10AD90000993069B4400E45A694B063CE4B20BAEAF
:10ADA000328807930294019100930599099BFFF75C
:10ADB000CBFC041E4CD1079B5E491B881A1D002D3D
:10ADC00030D14A80059B5B4C5A8963191A716B1C00
:10ADD0009BB2E318120A1A71162306A832881B18B0
:10ADE00079890598FCF74EFDFF21AA1C2E1D03351D
:10ADF0000B00059092B2B6B2ADB2002803D006ABFC
:10AE0000DB8AD9B21B0AA218651911712B714C4D3E
:10AE1000301D2A884949201800F076FB2B88F61847
:10AE2000B5B2A1E74988914207D17A8806995200C4
:10AE3000525AEB18053A9A42C4DC3E4C280061880D
:10AE400000F052FB207021007888FAF78BFED1E5E4
:10AE5000002DF2D13E89BFE6162606ABF61831006A
:10AE60003889FCF79BFC3D000400FA3500282DD002
:10AE7000037A9B060CD400227B893989788800925A
:10AE80003A000C32FFF7E8FB041E10D03E8915E0B3
:10AE90003088FFF741FB00281AD08368002B17D0B9
:10AEA0002100122278889847041EE4D0EEE72B7820
:10AEB000002B02D17888FAF765FE00262B78002B4C
:10AEC00000D097E5002C00D194E585E60124DDE76C
:10AED0000E24DBE7162506ABED1829003889FCF7B0
:10AEE0005DFC041E47D0037A9B0611D4154A7B886B
:10AEF0001188994203D01448814207D11380134B23
:10AF0000F2261D780023D9B2A94221D30924A1E752
:10AF10002888FFF701FB00282FD08368002B2CD056
:10AF20002100122278889847041EDFD092E7C0469D
:10AF30008464FF1F5468FF1F5668FF1F4869FF1F86
:10AF4000386AFF1F346BFF1FFFFF0000326BFF1FCB
:10AF500031005943546801336018615A0029D2D135
:10AF60003C0008342100F22200F0CEFA210078885B
:10AF7000FAF710FE3EE501246CE70E246AE71D4B4C
:10AF80001A887B889A4231D07888FAF70DFE31E52D
:10AF9000F223059851684343CD18C95A00291FD0A0
:10AFA0003B7A012B0BD16C88AB887888AA1D009462
:10AFB000FFF752FB041E02D000233B722E88F222C0
:10AFC0000021280000F0B8F900232B80059B0133F5
:10AFD000DBB20593084B05991B78064A8B42D7D8FC
:10AFE00001235B421380002CCED0F5E5002634000F
:10AFF0000596EFE7346BFF1F326BFF1F70B504003F
:10B000000E001500FFF796FA031E08D1310005481F
:10B01000FFF790FA03001120002B02D01C800020C3
:10B020009D7070BDFFFF0000F8B50B4F06003B7828
:10B030000D001400FF2B0ED00A2000F055F9011E60
:10B0400009D0B1230380002346800371C5800481A9
:10B05000387800F071FBF8BD1D44FF1FF7B50F00F5
:10B0600008A90600088809A90B240988002821D10D
:10B070000234022B1ED1557813782D021D432B006C
:10B080008B4301937334002B14D1FB6830001900FB
:10B090000093FFF74FFB019C85420BD02A00300044
:10B0A0000099FFF7ABFF041E04D12A003000798914
:10B0B000FFF7BAFF2000FEBDF0B50E7885B0039013
:10B0C0000AA805880120022E0DD14C6827786478E3
:10B0D00024023C43054FBC4205D10398DBB20196E4
:10B0E0000095FFF7BBFF05B0F0BDC0460229000088
:10B0F000034B10B51B68002B00D09847FEE7C046F5
:10B10000406BFF1F07B501A8FFF7F2FF044A05488F
:10B110000021121A00F070FAF8F7F4FAFEE7C046C0
:10B12000446BFF1F2044FF1F01B40248844601BC4A
:10B13000604700BF75A9000001B40248844601BC05
:10B14000604700BF291C000001B40248844601BCCE
:10B15000604700BF055E000001B40248844601BCA0
:10B16000604700BF810E000001B40248844601BC64
:10B17000604700BF8530FF1F01B40248844601BC10
:10B18000604700BF4938FF1F01B40248844601BC34
:10B19000604700BF5D17000001B40248844601BC4F
:10B1A000604700BF9536FF1F01B40248844601BCCA
:10B1B000604700BFB14E000001B40248844601BCA4
:10B1C000604700BF5139FF1F01B40248844601BCEB
:10B1D000604700BFF13AFF1F01B40248844601BC3A
:10B1E000604700BF453BFF1F01B40248844601BCD5
:10B1F000604700BFADAE000001B40248844601BC08
:10B20000604700BFEDA5000001B40248844601BCC0
:10B21000604700BF056A000001B40248844601BCD3
:10B22000604700BFCD4C010001B40248844601BC18
:10B23000604700BF090E000001B40248844601BC0B
:10B24000604700BF3D18000001B40248844601BCBD
:10B25000604700BF5549010001B40248844601BC63
:10B26000604700BF691F000001B40248844601BC6A
:10B27000604700BF0519FF1F01B40248844601BCA6
:10B28000604700BFC51D000001B40248844601BCF0
:10B29000604700BF2124000001B40248844601BC7D
:10B2A000604700BF8552010001B40248844601BCDA
:10B2B000604700BF0124000001B40248844601BC7D
:10B2C000604700BFC926000001B40248844601BCA3
:10B2D000604700BF434D010001B40248844601BCF1
:10B2E000604700BF1D3BFF1F01B40248844601BCFC
:10B2F000604700BF1D4D010001B40248844601BCF7
:10B30000604700BF6D30FF1F01B40248844601BC96
:10B31000604700BFB54C010001B40248844601BC3F
:10B32000604700BFA136FF1F01B40248844601BC3C
:10B33000604700BF091B000001B40248844601BCFD
:10B34000604700BF154D010001B40248844601BCAE
:10B35000604700BFF94C010001B40248844601BCBB
:10B36000604700BFC56D010001B40248844601BCBE
:10B37000604700BFAD32FF1F01B40248844601BCE4
:10B38000604700BF2951010001B40248844601BC56
:10B39000604700BF2D2EFF1F01B40248844601BC48
:10B3A000604700BF6571010001B40248844601BCDA
:10B3B000604700BF5147010001B40248844601BC08
:10B3C000604700BF1147010001B40248844601BC38
:10B3D000604700BFA946010001B40248844601BC91
:10B3E000604700BF3520FF1F01B40248844601BCFE
:10B3F000604700BFE928000001B40248844601BC50
:10B40000604700BFF54E010001B40248844601BC0C
:10B41000604700BF9537FF1F01B40248844601BC56
:10B42000604700BFC9A9000001B40248844601BCBE
:10B43000604700BFA54F010001B40248844601BC2B
:10B44000604700BF7918000001B40248844601BC7F
:10B45000604700BFC94A010001B40248844601BCEC
:10B46000604700BFB352010001B40248844601BCEA
:10B47000604700BF3119FF1F01B40248844601BC78
:10B48000604700BF4D1F000001B40248844601BC64
:10B49000604700BF156B010001B40248844601BC3F
:10B4A000604700BF5D34FF1F01B40248844601BC01
:10B4B000604700BFD532FF1F01B40248844601BC7B
:10B4C000604700BF4551010001B40248844601BCF9
:10B4D000604700BF851F000001B40248844601BCDC
:10B4E000604700BFED4A010001B40248844601BC38
:10B4F000604700BF090E000001B40248844601BC49
:10B50000604700BF5125000001B40248844601BCD9
:10B51000604700BFE94C010001B40248844601BC09
:10B52000604700BF350E000001B40248844601BCEC
:10B53000604700BFDD52010001B40248844601BCEF
:10B54000604700BFC521000001B40248844601BC29
:10B55000604700BF8D12000001B40248844601BC60
:10B56000604700BF3D4B010001B40248844601BC66
:10B57000604700BF6DBC000001B40248844601BCB6
:10B58000604700BF4550000001B40248844601BC3A
:10B59000604700BFC536FF1F01B40248844601BCA6
:10B5A000604700BFF30E000001B40248844601BCAE
:10B5B000604700BF3533FF1F01B40248844601BC19
:10B5C000604700BF3D39FF1F01B40248844601BCFB
:10B5D000604700BF2526000001B40248844601BC34
:10B5E000604700BFE117000001B40248844601BC77
:10B5F000604700BFE548000001B40248844601BC32
:10B60000604700BFB70E000001B40248844601BC89
:10B61000604700BF753BFF1F01B40248844601BC70
:10B62000604700BF311B000001B40248844601BCE2
:10B63000604700BF017F000001B40248844601BC9E
:10B64000604700BF5952010001B40248844601BC62
:10B65000604700BFDD66010001B40248844601BCBA
:10B66000604700BF5522000001B40248844601BC77
:10B67000604700BF0D31FF1F01B40248844601BC82
:10B68000604700BF3555000001B40248844601BC44
:10B69000604700BF753AFF1F01B40248844601BCF1
:10B6A000604700BFD949010001B40248844601BC8B
:10B6B000604700BF014C010001B40248844601BC50
:10B6C000604700BF9D3BFF1F01B40248844601BC98
:10B6D000604700BF093AFF1F01B40248844601BC1D
:10B6E000604700BFD91B000001B40248844601BC7A
:10B6F000604700BF613BFF1F01B40248844601BCA4
:10B70000604700BF456B010001B40248844601BC9C
:10B71000604700BF0D52010001B40248844601BCDD
:10B72000604700BF2146010001B40248844601BCC5
:10B73000604700BF8D1BFF1F01B40248844601BC57
:10B74000604700BF594F010001B40248844601BC64
:10B75000604700BF893BFF1F01B40248844601BC1B
:10B76000604700BF8B52010001B40248844601BC0F
:10B77000604700BFC939FF1F01B40248844601BCBD
:10B78000604700BF8939FF1F01B40248844601BCED
:08B79000604700BF1D4B0100E2
:10B798000200030004030503060307020803090364
:10B7A8000C030D001600090100000000E93A001121
:10B7B8001D3B00110000000002000000CAB7001184
:10B7C800192A0F181EFF4C0012190A00F15900001F
:10B7D800FD24000041460100D97B0011ED9B0011BA
:10B7E80041700011DD7900114953001189A9001138
:10B7F800F94E0011294000115941001100000000C4
:10B80800161600000200000018B80011F4FFF3FF3C
:10B81800D2FC000099420011000000000000000066
:10B828004449590042322E300030303230006769C6
:10B83800746875622E636F6D2F70767678004B454D
:10B84800590000000200000060B80011292A282AC7
:10B85800272A262A252A242A0A180000050000007B
:10B868001F501D10023CB40000011E002000000003
:10B8780009006000303132333435363738394142C7
:10B88800434445460000000001A0000000000000FD
:10B898006410B71DC8206E3BAC30D9269041DC76C9
:10B8A800F4516B6B5861B24D3C7105502083B8ED73
:10B8B80044930FF0E8A3D6D68CB361CBB0C2649B97
:10B8C800D4D2D38678E20AA01CF2BDBDFB349B5FBC
:10B8D800800000800010000000000000435C0011A0
:10B8E800CD720011675C0011D5760011EB5C001178
:10B8F800AB760011615D001181760011B35D001116
:10B90800497800111B5E0011497800114D5E001145
:10B9180003780011615D001139760011D95D0011BD
:10B92800E17700110000000000000000BF5E001178
:10B93800E1770011215F0011E5720011052A042A40
:10B94800012A002A022903280128002801180018C2
:10B958000000000000000000000000000000008758
:10B9680001010201020101020102030304010301B2
:10B97800010101010303020103000D000E00100084
:10B98800110013001401070108010A010B011C0131
:10B998001D02040205020702080219021A021C020B
:10B9A8001D03010302031700020100050400080734
:10B9B800000B0A001716001D1C01020101050401F5
:10B9C8000E0D011110011413011716011A190202A4
:10B9D80001020B0A020E0D021110021413021716AF
:10B9E800030504030807030B0A030E0D00010203F5
:10B9F80007090A0B0E0F101112141718191A1B1F1A
:10BA080020212200D1A200118DA300110000000006
:10BA18000200000056B9001100000000B9B0001182
:0CBA2800000000000200000054B90011F2
:020000041FFFDC
:1000000000000000913F0011D4B70011D2B70011D9
:10001000A861FF1F000000000000000000000000B9
:1000200000000000000000000000000000000000D0
:1000300000000000000000000000000000000000C0
:1000400000000000000000000000000000000000B0
:1000500000000000000000000000000000000000A0
:100060000000000000000000000000000000000090
:100070000000000000000000000000000000000080
:100080000000000000000000000000000000000070
:100090000000000000000000000000000000000060
:1000A0000000000000000000000000000000000050
:1000B0000000000000000000000000000000000040
:1000C0000000000000000000000000000000000030
:1000D0000000000000000000000000000000000020
:1000E0000000000000000000000000000000000010
:1000F0000000000000000000000000000000000000
:1001000000000000000000000000000000000000EF
:1001100000000000000000000000000000000000DF
:1001200000000000000000000000000000000000CF
:1001300000000000000000000000000000000000BF
:1001400000000000000000000000000000000000AF
:10015000000000000000000000000000000000009F
:10016000000000000000000000000000000000008F
:10017000000000000000000000000000000000007F
:10018000000000000000000000000000000000006F
:10019000F932FF1F5931FF1FC16601000000000046
:1001A000000000000000000000000000000000004F
:1001B000000000000000000000000000000000003F
:1001C000000000000000000000000000000000002F
:1001D000000000000000000000000000000000001F
:1001E000000000000000000000000000000000000F
:1001F00000000000000000000000000000000000FF
:1002000000000000000000000000000000000000EE
:1002100000000000000000000000000000000000DE
:1002200000000000000000000000000000000000CE
:1002300000000000000000000000000000000000BE
:1002400000000000000000000000000000000000AE
:10025000000000000000000000000000000000009E
:10026000000000000000000000000000000000008E
:10027000000000000000000000000000000000007E
:10028000000000000000000000000000000000006E
:10029000000000000000000000000000000000005E
:1002A000000000000000000000000000000000004E
:1002B000000000000000000000000000000000003E
:1002C000000000000000000000000000000000002E
:1002D000000000000000000000000000000000001E
:1002E000000000000000000000000000000000000E
:1002F00000000000000000000000000000000000FE
:1003000000000000000000000000000000000000ED
:1003100000000000000000000000000000000000DD
:1003200000000000000000000000000000000000CD
:1003300000000000000000000000000000000000BD
:1003400000000000000000000000000000000000AD
:10035000000000000000000000000000000000009D
:10036000000000000000000000000000000000008D
:1003700005B10011000000000000000000000000B6
:10038000000000000000000000000000000000006D
:10039000000000000000000000000000000000005D
:1003A0000000000000000000000000000D1BFF1F07
:1003B000000000000000000000000000000000003D
:1003C000000000000000000000000000000000002D
:1003D000000000000000000000000000000000001D
:1003E000000000000000000000000000000000000D
:1003F00000000000000000000000000000000000FD
:08183800506FFF1F4118FF1F54
:10184000024981F3088802F043FC0000506FFF1F3B
:1018500070B500241E491F4A1F484C6308CA1B0567
:101860001B0DE4188242F9D11C4B80228B630021AE
:1018700009201B4B920519621A4B1B4DDA671B4B53
:10188000DA688243DA609A68194802409A60112047
:10189000296002F0B9F8112002F096F880226B6CF2
:1018A000112093436B64EE23DB006343114A1B0C4E
:1018B00013840122104B9A7401F004FC0F4B1B7827
:1018C000002B04D10E4B1021187802F0D1F970BD15
:1018D000000005408805054000060540FF010000A6
:1018E00000F0004004E100E0003800403CF000401F
:1018F000FFDFFFFF2061FF1F1462FF1F4A64FF1F0D
:101900004862FF1F10B502F0D3FA072804D012284E
:1019100008D0022808D010BD044A0420136B0133FC
:101920001363F8E70220F6E71420F4E72C65FF1FA5
:10193000F8B507000C0026002500503630785135E8
:10194000002804D10300287058342370F8BD29788A
:10195000CA00481E8141A3183800A25C5B68C9B266
:10196000FFF7D0FF00280DD12B78DA00A218013341
:1019700050602B703378044A013B3370136A013393
:101980001362D8E70123DFE72C65FF1F5C23434385
:10199000074910B5C9180B0058331B78012B05D126
:1019A000FFF7C6FF034A936A0133936210BDC04636
:1019B0006065FF1F2C65FF1F10B502F059FB064A3A
:1019C0000121130010CB4942D967044B136002F088
:1019D0005FFA200010BDC04600E100E010001000DA
:1019E00010B5040002F044FB024B1C6002F050FAF8
:1019F00010BDC04600E100E0431E5A425341A02200
:101A0000F0B5D2015B421340154D164A40019B18B8
:101A10002A18127E8BB00191002A1BD01A000832BE
:101A2000D46F0022E6B206AFE4B294420EDC28186E
:101A3000C369002B08D0019902AA117106AA049269
:101A400002AA167303A898470BB0F0BD1978B954D1
:101A50000132EAE71A7D1A7806AB01261A70E6E72A
:101A6000EC67FF1F00400040F0B5254B040040012B
:101A7000C25C85B0002A2BD01A18117E002927D00D
:101A8000917E002924D01179022921D11689D78885
:101A9000D168F51BADB22A1C102D00D9102292B2CC
:101AA000BE4217D11818012303710023C269C380F5
:101AB00003819A4206D068460321037301710293A1
:101AC00001A890470820002C00D0192001F0FAFA54
:101AD00005B0F0BD013C65426C41A0256442ED01BA
:101AE0002C40084D1B186419074D0633013A92B279
:101AF000AA42EDD01888461C1E80085C2070F5E7CD
:101B0000EC67FF1F00400040FFFF00000F220E4B5C
:101B100010B59868104002380A280BD802F02AF84D
:101B20000D0A0B0A0A110A0A0A0A060002210020FD
:101B3000FFF762FF10BD0121F9E70020FFF794FFD6
:101B4000F8E7DB6FF6E7C046004000400F220E4B7F
:101B500010B59868104002380A280BD802F00AF82D
:101B60000E0A0B0A0A120A0A0A0A060002210120BA
:101B7000FFF742FF10BD01210800F9E70120FFF740
:101B800073FFF7E7DB6FF5E70090004013B5334CC8
:101B90002378072B3DD8324B1A78324B002A39D1A3
:101BA0008022196852020A431A60252001F0ECFED7
:101BB00020232D4A11680B43802113606B460422B9
:101BC000C90508680733104228D080210422C905BE
:101BD000C86810422ED080212020C905CA688243DF
:101BE000CA6014221A701A78002A2FD18021C905E0
:101BF000C86820320243CA6014221A701A78002A78
:101C000028D11A4B1A7D22785A601D221A70593237
:101C1000DA6013BD1A6816490A40C5E7086802432E
:101C20000A6014221A701A78002ACED01A78013A63
:101C3000D2B2F7E7C8680243CA6014221A70197852
:101C40004A1ED2B21A700029F9D1C4E71A78013AB3
:101C5000D2B2C7E71A78013AD2B2CEE75843FF1F93
:101C60002044FF1F3CF000405043FF1F0020004075
:101C7000FFFFFEFF564B70B51B68012B03D1554A81
:101C8000936D0133936502F013FA534B534A186076
:101C9000534B544C1A600123534A1360534A136048
:101CA0002378002B06D006225149524802F010F941
:101CB00000232370504A514B10681B78C1B2002B8F
:101CC0000ED14F4CC0B223785BB2002B4FDB237890
:101CD00024785BB264B21B0424021B191B18136026
:101CE0000B1C50294ED95023464A47491078DBB285
:101CF000FF2202284BD10868444C454D267890437A
:101D00002A78964254D9227824782E78023B5D10A6
:101D1000A31B6B435201D31A10335B1118430860A5
:101D200001F0FEFF031F012B45D83A4B1B78002B17
:101D300006D0394B1B78002B02D0002001F060FF49
:101D4000A122364B92009978354B4A431B689B1869
:101D5000832292009B181B78033B012B03D8AF20F2
:101D6000400002F0F5F801222E4BDA8270BD237894
:101D700024785BB264B2FF33FF341B0424021B19C6
:101D80000138ABE7CAB2022AAED20223ACE7086838
:101D9000254C264D267890432A78964208D92278F9
:101DA00024782D78023B5B10641B63435201B2E739
:101DB0002378DBB2B2E70228D5D11D4B1B78013B5B
:101DC000022B03D91B4B1B78022BCCD16C20C8E70C
:101DD0009809FF1FFC0FFF1F7864FF1FFF3F0000E3
:101DE000141003407C64FF1F0C10034000100340DC
:101DF000D50BFF1F7211FF1FB40003408C09FF1F9A
:101E0000680AFF1F490AFF1F94000340460AFF1F8C
:101E1000470AFF1FF908FF1F2209FF1F300DFF1F90
:101E20003409FF1FBC0BFF1F440AFF1F450AFF1F99
:101E30001C09FF1F2309FF1F10B502F081F80022C3
:101E4000014B1A8010BDC0467464FF1F10B502F02C
:101E500037F9A121054A89009478054A614312683F
:101E6000044B5218528C1A8010BDC046300DFF1F13
:101E70003409FF1F7464FF1F10B50D4B0D4A99788C
:101E8000A1239B004B431268D218531DD97F0A4BE4
:101E90001B88994209D2441C07D0C82805D0D269B2
:101EA0005B1A5A43054B5343C01801F029FF10BD7C
:101EB000300DFF1F3409FF1F7464FF1F7102000003
:101EC00070B5244D2B68002B28D001F0B1FF2B6892
:101ED000D8402B680400002B27D001F019FF2B6895
:101EE000D8401D4B1D4A9978A1239B004B43126893
:101EF000D118D25C91239B00002A20D0CA5801320D
:101F0000CA50174B17491B680868834214D3D23B49
:101F1000181A012A1AD0144B186070BD01F088FFFE
:101F2000124B196801F0C4FED3E701F0F1FE0F4B2C
:101F3000196801F0BDFED4E70D495B18E8E7CA5007
:101F40000C4B1B68DB68E418201AE4E7F530FF301F
:101F5000E1E7C0461C08FF1F300DFF1F3409FF1FBB
:101F60009C09FF1F7864FF1FA009FF1F1808FF1FAF
:101F70002DFF3F008064FF1F70B504000D0028296D
:101F800016D10300A433C2881B889B1A0B4A9BB24C
:101F900093420DD906006A3605223100653002F001
:101FA0004FF8002804D13100200001F009FE70BD77
:101FB0002900200001F0F4FFF9E7C046FE7F000091
:101FC000F8B50500012002F05BF8134CA36AA26A81
:101FD0009342FBD1114E336002F022F81049030006
:101FE00008601048426894460F4A17680022BC45B2
:101FF00001D24268BA1A0D4802603268AD18A422B4
:10200000E562606A520302436262094A1278002A5A
:1020100001D00F3B0B60F8BD00F00040340AFF1FF9
:10202000E408FF1F28100040180AFF1F1C0AFF1FAA
:102030001C09FF1F70B580241025E405A3682B43FD
:10204000A36001F0A5FEA368AB43A36070BD0000D0
:10205000F7B5160080221C001023D205019191686B
:1020600005000B43936000225A4BD7301A6001F0F1
:102070007FFE9D232A002F009B00EB58CA320121CE
:102080000092FC37002B01D00021009A386801F043
:1020900047FF2900009BCB311A784F4BD3351A608C
:1020A0004B780A781B0213438A7812041A43CB78C0
:1020B0001B061343494A1BBA13604B790A791B026A
:1020C00013438A7912041A43CB7931001B06134358
:1020D000434A1BBA13606B782A781B021343AA7811
:1020E00012041A43EB781B0613433E4A1BBA1360D3
:1020F000019A330213433C4A13603C4B22001B1BE2
:102100009C4603293DDCB3089A0013005142B21AE1
:10211000032A46D1354AE018511A827840781204D1
:1021200000020243E05C043302430A600022FF2BFA
:102130004BDDF0222E4B12011A600F222D4B1A603C
:102140002D4A1368002BFCD00023224A2749136034
:10215000091B321D0B191B68043A180A23706070A2
:10216000180C1B0EA070E3700434002AF2DC8022ED
:1021700010213B68D20501333B6093688B43936029
:10218000F7BD6346D578981893782D061B042B432A
:10219000157804392B43557804322D022B43036004
:1021A000AFE7022A0AD1114AE05C511AE2185278CC
:1021B000120202430A6004339BB2B7E7012AB5D189
:1021C0000A4A521AE15C1160F5E7084959180A6099
:1021D0000433ACE7000004403C00044038000440F5
:1021E00034000440300004400C000440000104406E
:1021F000040004401000044014000440F7B515002A
:1022000080221C001023D2050091916807000B4327
:1022100093600023654AD730136001F0A9FD9D2328
:102220003E009B00F9583B00CA363200FC330029BF
:1022300000D07FE0586801F073FE390032785C4BC3
:10224000CB311A604B780A781B0213438A78AC466C
:1022500012041A43CB78281D1B061343554A1BBA98
:1022600013604B790A791B0213438A7912041A43CB
:10227000CB791B061343504A1BBA13604B7A0A7A78
:102280001B0213438A7A12041A43CB7A21001B06DD
:1022900013434A4A1BBA1360009A2B021343484A5D
:1022A00013602200474B1B1B0093009BCE785B18EA
:1022B00001938B7836061B0433430E78043833437E
:1022C0004E78043136023343019E33600328ECDC40
:1022D0000321A808431C9B002940800003292BD11F
:1022E0003849E5185E18A9786D78E35C09042D0279
:1022F000294319433160030008330021FF2B2DDDF2
:10230000314B324919600F21314B196001232749A4
:102310000B60304B19680029FCD006211B680B406C
:10232000042B20D080220020D20593680A318B43F1
:102330009360FEBD01217DE7022908D121495D1886
:10234000E1184978E35C090219432960D3E70129C0
:10235000D3D11C495918E35C0B60CCE71948181815
:1023600001600433CAE7002310490B606346002B69
:102370000CDC3B00FC335A68102101325A60802289
:10238000D205936801208B439360D2E7009B9B1892
:102390001B68190A13705170190C1B0ED37004239B
:1023A0005B4291709C440432E0E7C0460000044068
:1023B0003C00044038000440340004403000044035
:1023C0000C0004400001044004000440080F000019
:1023D000100004401400044070B5061E19D00222FB
:1023E0005A4B9B799343012B13D1594B1A78FF2AEF
:1023F0000FD15A78FF2A0CD19A78FF2A09D1DA78BE
:10240000FF2A06D11A79FF2A03D15B79FF2B00D16D
:1024100099E0504B0C201A78012A08D000224E4D2A
:102420001A7029780B00093B042B01D8212070BDBC
:102430004B1F012BFAD9454CA37B042B00D982E01A
:10244000A279032A00D97EE09A1ED2B2012A02D8CC
:1024500060881F2877D9002E56D0012E73D1A0880E
:102460000128E3D0002907D1581E032803D801F022
:1024700081FB121715122E702978481E032811D8D7
:102480000025364B1D602823237501F0E1FBA8428F
:1024900027D0A580CAE702212970EDE70421FBE7D8
:1024A0000321F9E707390129C0D82D490968C96A0C
:1024B0008906BBD52B4908780028B7D1012A01D954
:1024C000002BB3D102230B708021274D26338901C5
:1024D0002878237501F094FD80212878890101F086
:1024E000C7FB0123A380214B1B78002B0AD0FA22C3
:1024F00080211F4B92001B8809025A431A4B1878FF
:1025000001F0C6FD002092E701F0B2FD2B78A68015
:10251000073B012B03D917482E7001F0C1FD114B69
:10252000114C1A78002A06D08021002220788901D7
:102530001A7001F065FD01F0ABFC802120780902E2
:1025400001F05EFDDEE7122071E7C046A60BFF1F1B
:102550006B09FF1F1A09FF1F1C09FF1F4809FF1FF6
:102560008064FF1F2309FF1F1B09FF1F2109FF1F95
:102570002C09FF1F0010004010B5002901D001F008
:1025800047FD10BDF7B5604B01919978A1239B00E1
:102590004B435E4A060014681022E418D6235B0001
:1025A000E0583623FF33E35C00279343222B41D1CD
:1025B000574B0F3A1A600760012501F0D1FB019BD0
:1025C0001880E8235B00E35C002B01D0B34258DDA8
:1025D0000023504FFB70AD33FF33E3581A68002AD5
:1025E00003D09B88DB439B071DD03823FF33E35C7C
:1025F000002B18D09B235B00E35C002B13D1D1335D
:10260000FF33E35CB3420EDAA4235B00E15AE01827
:10261000090A023101F014FB23000122FE33013EBE
:1026200001351A87FA70E8235B00E35C002B2AD09F
:10263000A8B2FEBD03683D00002BBED081880430E7
:10264000090A023101F0FCFAD6235B00E3581F604F
:10265000B2E72300B133BA00FF33985801378188BD
:102660000430090A023101F0EBFAE8235B00E35C75
:10267000BB42EEDCE822F61AED1800235200A35408
:10268000A6E70027F1E7200001F032FC00281FD068
:10269000002E1DDD7319882647190193B60020000E
:1026A00001F06EFB5A3080002018406801358188A7
:1026B0000430090A023101F0C3FA200001F078FC6D
:1026C000A3590133A351BD4202D0019B9D42E6D1E3
:1026D000114BE35C002BABD095239B00E35C002BFC
:1026E000A6D00E4BE15A0029A2D00D4AA35C994214
:1026F00002D90133A3549BE700231A212000A354DD
:1027000001F01EFB94E7C046300DFF1F3409FF1F88
:1027100000140340E010FF1F5A0200007202000084
:102720005E0200000D4970B54A6E0D4CD2038B69F4
:10273000D20BA24206D80B4D0224AA4204D901F0C2
:1027400067FA70BD02246442E21815007E24254019
:102750002242F4D0A3432B438B61F0E700F000400A
:102760000A200000FC1C0000F8B51D4B1D4F1A7814
:10277000002A10D1BA7B002A02D101321A7003E07C
:10278000032AFAD0022AF8D001F062FA00220120CE
:10279000154B1A70F8BD154B154D1C68154B9E78DE
:1027A00001232B702878C0B200F09EFBBB7B002B6E
:1027B0000BD101F0ADFBA1239B007343E4188323ED
:1027C0009B00E41823782B70E4E7032B02D101F07F
:1027D000FFFAF0E70020022BDCD101F061FAEAE712
:1027E0001C09FF1FA60BFF1F2309FF1F3409FF1F32
:1027F000490AFF1F300DFF1FF0B587B00EAD2F78CF
:102800000FAD2D780593AC46634614000E4D0CAA0F
:1028100012782E7803930D9B009201932200059B62
:10282000029701F0C5F92E70012C01D0042C08D1BB
:10283000802206498B889343054A1278D2011343BC
:102840008B8007B0F0BDC0461C09FF1F6C11FF1F35
:102850007809FF1F0B001B3B70B504003020E02BF4
:102860000DD81300E025493BFF3B9BB2ED00AB4286
:1028700005D8034B200019825A8201F0E9FB70BD94
:102880008410FF1F10B501F013FC054B00205B689E
:10289000052B04D9034A5268D20200D4980810BD0F
:1028A00000100040FCE100E070B501F0E1FB0D4BD1
:1028B0001B68FC33DC691D6AFFF7E4FF641984427E
:1028C00004D2094B01241B68002B07D004220024EA
:1028D000064B1A70064A93690133936101F0D8FAE6
:1028E000200070BD8064FF1F9809FF1F2309FF1F90
:1028F000FC0FFF1F70B50C4D2B68FC335C6A01F0B8
:10290000B7FBFFF7BFFF2B680025FC339B6AE3187A
:10291000834204D2054B1B68AB4200D1051B01F07A
:10292000B7FA280070BDC0468064FF1F9809FF1FDA
:10293000D722044B92009B5810B5002B00D098472B
:1029400010BDC0460000FF1F10B501F0FBF8FFF7F7
:10295000EFFF2749274BCA6D274C1A4084235B00A1
:102960001343CB65254B1B68186A01F089FB244B88
:10297000244A1A60244B254A1A60A022244B520094
:102980001A60244B187801F013FA2000224901F054
:1029900077FA0023A3600233A360204B2049236011
:1029A00003232048A36001F06BFA10221E4BFF2086
:1029B0001A60802252031A60802292031A608022D9
:1029C00012041A6001F01CF9012001F0C1F9FA208B
:1029D000400001F0ADFA582001F0BAFA134801F0B6
:1029E000FFF8012001F06CF9072001F0F9FA10BDA1
:1029F00000F0004000FEFEFF141000408064FF1F46
:102A0000000003400180063DBC0003403408000084
:102A1000A40003404A0AFF1F71020000C30900001E
:102A2000FFFF3F002810004000E100E0307500008B
:102A3000674E336888331B6883F3088801F0B0F968
:102A4000644A6549136800200B401360634B644A75
:102A50001B68934200D1A6E001F022FA0221614AEC
:102A600013688B431360FFF76FFF5F4B5F4C187861
:102A7000C0B201F035F90023A3600233A3605C4BC0
:102A80000120236001F0FCFA0323A36001F0C8F8E1
:102A9000040001F00DFB050001F0C2F8554B186071
:102AA00001F0CEF9544B1968621A531EA14200D2AC
:102AB00013008022D203934201D39B029B0A326807
:102AC000D16AC90700D471E04C491C0C09689BB25B
:102AD0004C4359432402090A641803264849FC322E
:102AE00093680A6847489B1A474A0768126847492B
:102AF0009B18474A9A1833409208DB190A60036012
:102B0000042B03D9013233400A6003600E68414947
:102B1000A619300001F0CCF83F4F3E493B68C3187E
:102B20003B603000019301F003F93C4E3068081817
:102B300038493060884205D9019B01333B6001F080
:102B4000F7F8316001F054F8354B1B78002B0DD0AD
:102B500001F0AEFA334B621B196812188A4232D266
:102B60004919091B091A304801F08AF92F4E337AA6
:102B7000002B0ED001F09CFA621BF16812189142F2
:102B800024D94919091B091A294801F079F90023A8
:102B90003372284B83F3088801F092F9002001F08A
:102BA0007FF901F015F801F07BF95CE7DC01990091
:102BB0000234641A5900641A09214B438033CB4014
:102BC000A408E41889E7FA218900CCE71A49DBE771
:102BD0008064FF1F1CF00040FFFFC1FF0C0AFF1FB5
:102BE000B641210310000040490AFF1F14100040A5
:102BF000C3090000100AFF1F340AFF1F380AFF1F15
:102C0000200AFF1F280AFF1F1C0AFF1F240AFF1F9C
:102C1000C4090000710200006008FF1F2C0AFF1F9A
:102C20001C09FF1FE408FF1F00100040740BFF1F6A
:102C30003C10004000000020DC050000A022054BF5
:102C400092009B5810B5002B01D0984710BD01F0A1
:102C5000EFF9FBE70000FF1FA122054B92009B58F4
:102C600010B5002B01D0984710BD01F0E1F9FBE74A
:102C70000000FF1FA222054B92009B5810B5002BAD
:102C800001D0984710BD01F0D3F9FBE70000FF1F0A
:102C9000A322054B92009B5810B5002B01D09847FA
:102CA00010BD01F0C5F9FBE70000FF1FA422054B92
:102CB00092009B5810B5002B01D0984710BD01F031
:102CC000B7F9FBE70000FF1F70B501F0F1F94F4BBA
:102CD000186001F07DF90400C30702D401F0A0F8E8
:102CE00070BD00224A4B1A604A4B187801380428FC
:102CF00029D800F03FFF0320181C2400200000F01A
:102D0000C7FF0128ECD0444C2378042B6ED101F08E
:102D1000F7F80028E4D001F07BF8582001F018F90A
:102D200002232370DCE7200001F022F9E9E720000C
:102D300001F026F9E5E7200001F092F9E1E7200033
:102D400001F086F8DDE700F0EBFF0500012808D16F
:102D5000324B1B78053B012B03D82000FFF76EFF99
:102D6000D1E72D4B1B78022B01D0052B20D1022D52
:102D700028D12B4B9B7BAB431CD12000FFF76CFF72
:102D8000264B18780128BED16405BCD424492522DD
:102D90004B7B034205D1233A13405A425341263319
:102DA0001A000B7D9342AED9322001F059F8AAE700
:102DB000022D07D1194B1B78052B11D12000FFF7ED
:102DC00059FFDDE7012D0BD1012B03D12000FFF7C7
:102DD0005FFF98E7062B03D12000FFF767FF92E71C
:102DE000200001F025F9022D8DD1C9E7032B04D174
:102DF0000C4B987C01F03CF872E7072B00D06FE792
:102E0000094B987B00F0ECFF6AE7C0469C09FF1F66
:102E10009809FF1F9009FF1F2309FF1F1C09FF1FAF
:102E2000A60BFF1FBC0BFF1FD40BFF1FFA210A4B81
:102E30000A4A49001A640A4A5A500A4A04395A503E
:102E4000094A08319A64094A5A50094A5C315A5071
:102E5000084ADA667047C0460000FF1FF927FF1FC7
:102E6000F528FF1FA928FF1FD923FF1F6927FF1F70
:102E7000791EFF1F4D1EFF1FF7B50B0CFF27012208
:102E8000009300233C001E001D009446019089B26F
:102E900062469A401000084018413618B6B2FF2F1B
:102EA00002D1012E00D19FB2009802401A41AD1804
:102EB000ADB2FF2C02D1012D00D19CB20133102BF9
:102EC000E6D10320012E07D1012D04D1019B24015D
:102ED000E4191C700138FEBD102EFCD10238102DF3
:102EE000F9D00230F7E700008023F7B59C46264B67
:102EF000264F01932649274A274D284C284B022864
:102F00001AD1604638600868264E30408026360365
:102F10003043086001990978002909D11660224AD6
:102F20002A60224A2260E02219689143A03A1BE0FD
:102F30008021C9021160F2E766463E600F68194EB3
:102F40003E408027FF023E430E6001990978002928
:102F50000DD1176001280ED1154A2A60154A22604A
:102F6000E02219689143C03A0A431A60F7BD8021F4
:102F700089021160EEE7E0210F4A02432A600F4AFE
:102F800022601A688A43F0E74B0AFF1FE000034003
:102F9000D80003409000034000000340500003406D
:102FA00040000340FFFFE3FF0280063D804508220A
:102FB0000180063D80660822008006988055082220
:102FC000F8B51E4B80261A680020140034403242A7
:102FD00032D11A681A4F32431A6001223B68063018
:102FE00093433B6001F04CF80122164D2B681E43C1
:102FF0002E603B680A2613433B608027BF00124BBC
:103000001B683B4211D1013EF6B2FF2E09D17E2250
:103010000E4B1C682B68E40B1440934323432B6036
:1030200005E0082001F02CF8E9E7002EEFD180221E
:103030002B68600893432B60F8BDC046C4F0004085
:103040005CF0004018F0004068F0004060F0004084
:1030500010B500F04DFE01215820034A00F040FF5A
:10306000FFF7AEFF10BDC046600AFF1F10B5782203
:103070000021034800F02CFE00F0BAFE002010BD35
:103080007467FF1F70B5040000F0F2FF00230C20EE
:103090000B4A010059438D18515C00290DD0A14203
:1030A00008D1012300246B7000F0AAFE00F0F0FEAE
:1030B000200070BD01330A2BEBD11224F6E7C04685
:1030C0007467FF1F70B5040000F0D2FF00231900E1
:1030D0001D000D4A1078002806D0A0420CD1557072
:1030E00001310C320A29F5D1002B0AD100F080FE03
:1030F00000F0CEFE002070BD5078461EB0411B1877
:10310000EEE700F07DFEF3E77467FF1FF7B50400FC
:103110000C20002384460E4D019267465F43E85D14
:103120007E19A04212D000280BD10A4B9C46624661
:103130001B7808331370019B70707C557160B3600D
:10314000FEBD01330A2BE8D10320F9E70720F7E79A
:103150007467FF1F7067FF1F8020F8B5484BC005DC
:103160001B68C1248360474BFF251A680123134362
:103170004361454BA4001A68444B40211A60444BFC
:103180001A68444B1A60444B1A59AA431A51C52273
:1031900092009E58AE433143802699509F583F4934
:1031A000F6010F403E439E509E5880273602360A55
:1031B0003043985080201A5900020A4002431A51A5
:1031C00004341A59364E3F04324080263A431A518D
:1031D0001A5936061202120A32431A5108341A5981
:1031E00080260A4002431A51C32292009F58B446D7
:1031F000AF4337439F509F58294E0F4007439F507E
:103200009F58374080263604374380269F509F586A
:1032100036063F023F0A37439F50C0221F59AF4333
:103220003A431A511A591202120A1643C6221E5163
:1032300092009C58AC4365462C439C509C580025FA
:103240000C4020439850C72080001A58154C11405C
:10325000C02212020A431A50134B1B78DB08AB4200
:1032600001DC0020F8BD2378002B06D0A368002BDA
:1032700000D0984701350C34EEE71220F2E7C04643
:103280005443FF1F5043FF1FB0F000406C67FF1F07
:10329000B4F000406867FF1F00E100E0FF00FFFF9F
:1032A000FFFF00FF7467FF1F7067FF1F030010B56B
:1032B0001F2809D8072200201340072404490A7850
:1032C000A24313430B7010BD00230620F5E7C04650
:1032D0007067FF1F054B06491B780A6805485B07A6
:1032E00002401B0B134300200B6070477067FF1FE9
:1032F0001CF00040FFFFC1FF70B50C25FFF7EAFF8F
:103300000A4B1C780A4BE4086543ED18002C01D1E8
:10331000200070BD2B78002B06D06B68002B00D0EE
:103320009847013C0C3DF1E71220F2E77067FF1F60
:103330006867FF1F70B50D00040000F099FE402182
:103340000F4AAD00136865198B431360AC4208D176
:10335000002202200B4B1A600B4B186000F068FC37
:10336000FEE7637801212078002B00D0032100F0D4
:103370000FFE6178207800F073FC0434E6E7C04665
:103380001CF00040C4F00040C0F000401FB5002118
:1033900002220B0001910091052000F0E1FD0223C3
:1033A0000B490A681A42FCD120230393039B5A1E3F
:1033B0000392002BFAD1074A1368002BFCDA0B2486
:1033C0006C442000012100F013FE207804B010BDF1
:1033D00090C8004000C8004013B504000A4B019398
:1033E000019B002B01D1112016BDFFF7CFFF230059
:1033F0000340044205D0052000F042FE019B013B42
:10340000EDE71800F0E7C046FFFFFF0707B500F043
:103410002FFE80220821D205936A0191002B01D151
:103420000739916202210C4A11600199481E0190EE
:103430000029FAD103311160053101910199481E2B
:1034400001900029FAD11160002B02D18022D2050F
:10345000936200F01DFD07BD00C00040F0B52D4C8B
:1034600089B02378002B4FD1FEF7A6FA02232A4F0A
:1034700003903A681A42FCD120230693069B5A1EF9
:103480000692002BFAD1254E3368002BFCDA01207E
:10349000FFF7A2FF011E02D0112009B0F0BD03000A
:1034A00003220190009005AD9F2000F059FD0321FB
:1034B000280000F09DFD02233A681A42FCD1202327
:1034C0000793079B5A1E0792002BFAD13368002BF3
:1034D000FCDA0120FFF780FF0028DDD10398FEF71A
:1034E0007FFAAA786B7811041B020B4329780B43EF
:1034F00063601300113B0A49052B07D80123934051
:10350000A3600B60012323700020C6E780231B0308
:10351000F6E7C0463C43FF1F90C8004000C800408B
:103520009808FF1F1E4B30B55A6818781D4B85B0A0
:10353000D31859424B4101210093002300F040FD74
:10354000194B1A4A02259A6300221A6510325A65ED
:103550008022C4219D65164B1648D202DA67890085
:103560004258154B80241A4080231B0413434350B8
:10357000642341200393E40500F006FA402000F0A4
:1035800003FA6562039D6B1E0393002DFAD103239A
:103590006362FFF73BFFA562FFF760FF05B030BD38
:1035A0004843FF1F95FFFEF700C80040050001FFDC
:1035B00004E100E000E100E0FFFF00FFF0B585B0AE
:1035C0000700FEF7F9F9022305002D4C22681A4284
:1035D000FCD120230093009B5A1E0092002BFAD1AD
:1035E000284E3368002BFCDA0120FFF7F5FE002897
:1035F00003D01124200005B0F0BD234B236002232B
:1036000022681A42FCD120230193019B5A1E019289
:10361000002BFAD13368002BFCDA0120FFF7DCFE27
:103620000028E6D1194B1F60022322681A42FCD100
:1036300020230293029B5A1E0292002BFAD1336878
:10364000002BFCDA0120FFF7C7FE0028D1D1104B78
:103650002360022322681A42FCD120230393039B98
:103660005A1E0392002BFAD13368002BFCDA01209A
:10367000FFF7B2FE041EBCD12800FEF7B1F9B9E78E
:1036800090C8004000C8004001000006A8C80040E3
:103690000180000110B50020FFF790FF10BD000071
:1036A00010B5064B18705960FFF73CFF002113203E
:1036B000034AFFF72BFD002010BDC0464843FF1F03
:1036C0002535FF1FF0B5040085B003920291FEF787
:1036D00073F9882263035B0B52051A438023DB05D1
:1036E0009D6A8023274F0092BA68002601901B0331
:1036F0009A420CD9F82326001B041E401C4206D017
:103700008022214B52025E6219680A431A60002D22
:103710000BD100F0ADFC02221C4B1A608023DB05AC
:103720005A62013A9A6200F0B3FB0023039A934273
:1037300020D1002D0AD100F09BFC144B03221D6008
:103740008023DB055A629D6200F0A2FB8023BA68E9
:103750001B039A4208D9002E06D000220A4B0C49BE
:103760005A621A680A401A600198FEF739F9002077
:1037700005B0F0BD009A0299D2181278CA540133EC
:10378000D4E7C0463C43FF1F00C8004000C00040D3
:10379000FFFFFEFFF0B587B0029103920400FEF731
:1037A0000BF9019000F064FC802302250122234ED6
:1037B000DB0535605D629A6200F06AFB204F3B6872
:1037C0002B42FCD120230493049B5A1E0492002B0D
:1037D000FAD11C4D2B68002BFCDA0120FFF7FCFD11
:1037E000002802D0112007B0F0BD2000039A0299F2
:1037F00000F0E6FA022304003A681A42FCD12023C2
:103800000593059B5A1E0592002BFAD12B68002BBD
:10381000FCDA0120FFF7E0FD051EE3D100F028FCF3
:1038200080230322DB0535605A629D6200F030FB85
:103830000198FEF7D5F8E0B2D5E7C04600C00040D9
:1038400090C8004000C80040F0B5802489B0060050
:10385000FEF7B2F8E405A36A02250393029000F094
:1038600007FC0123304F3D606562A36200F010FB4E
:103870002E4C23682B42FCD120230593059B5A1E16
:103880000592002BFAD12A4D2B68002BFCDA01207F
:10389000FFF7A2FD002803D01124200009B0F0BDDD
:1038A000244B2360022322681A42FCD12023069372
:1038B000069B5A1E0692002BFAD12B68002BFCDACD
:1038C0000120FFF789FD021EE6D11B4B03211E607C
:1038D000030001900090202000F042FB02232268A8
:1038E0001A42FCD120230793079B5A1E0792002BF4
:1038F000FAD12B68002BFCDA0320FFF76DFD041EC4
:10390000CAD100F0B5FB80230322DB053C605A627C
:103910009C6200F0BDFA039B002B01D1FFF776FDFE
:103920000298FEF75DF8B8E700C0004090C800407C
:1039300000C800400100000694C8004007B500021E
:1039400001910422000A01A9FFF724FF0EBD000027
:1039500073B5050005240B4AA3005B429B18196848
:103960006B46DE1D3000FFF787FA022804D133785A
:103970002B55013CEFD276BD052CFCD00128FAD1A5
:103980000230F8E7140900111F2807D8012380220C
:103990008340D20591680B43936070473F2808D855
:1039A0000123802220388340D20551690B435361A3
:1039B000F3E75F28F1D80123802240388340D20505
:1039C000116A0B431362E8E71F2807D80122802100
:1039D0008240C9058B6893438B6070473F2808D8A5
:1039E0000122802120388240C9054B6993434B61F5
:1039F000F3E75F28F1D80122802140388240C905D1
:103A00000B6A93430B62E8E71F2810D8802302005B
:103A1000DB05153A1968012A06D82022914319605E
:103A200019680A431A60704701228240F6E73F286E
:103A300011D880230200DB05353AD968032A06D85D
:103A400010229143D960D9680A43DA60EBE701227A
:103A500020388240F5E75F28E5D842238022181AF3
:103A6000413B8340D205516A99435162516A0B43ED
:103A70005362D8E710B50400012813D1A0221849D9
:103A800092050B685B015B0913430B60154B164AEB
:103A900019681140154A0A431A60402219680A43FE
:103AA0001A6010BD0028FCD101000A2000F0E8F8DF
:103AB00021000B2000F0E4F8C0220A4B92001968A4
:103AC0000A4340211A601A688A431A60B0220449E6
:103AD00012060B685B015B0913430B60E1E7C0460C
:103AE00014F000401CF000407F00FEFF80FD01004C
:103AF00072B6074A1368013313600422054B1A603B
:103B00000023054A13608022D2055360FEE7C046B9
:103B10007808FF1FC0F00040C4F0004005490B6862
:103B2000002B05D1044A0A6004490A60044A136064
:103B30007047C046140AFF1F841E0000380AFF1F8A
:103B4000C4F000400023034A1360034A1360034A91
:103B50001360704754F0004040F1004044F10040D1
:103B600002B4714649084900095649008E4402BC16
:103B70007047C04602B4714649084900095C4900D3
:103B80008E4402BC7047C04603B4714649084000E9
:103B90004900095E49008E4403BC704703B4714676
:103BA000490840004900095A49008E4403BC704747
:103BB00001B40248844601BC604700BF9D6A000012
:103BC00001B40248844601BC604700BF85C10000C3
:103BD00001B40248844601BC604700BF8552010021
:103BE00001B40248844601BC604700BF8D1101004A
:103BF00001B40248844601BC604700BFD5440100BF
:103C000001B40248844601BC604700BFED6B01006F
:103C100001B40248844601BC604700BFD1AE000039
:103C200001B40248844601BC604700BF156B010027
:103C300001B40248844601BC604700BFA1AF000048
:103C400001B40248844601BC604700BFC1150100B1
:103C500001B40248844601BC604700BFA9D80000F7
:103C600001B40248844601BC604700BFB5B2000001
:103C700001B40248844601BC604700BF0D520100F8
:103C800001B40248844601BC604700BF9D9D0011FD
:103C900001B40248844601BC604700BF0134010002
:103CA00001B40248844601BC604700BF19FA000015
:103CB00001B40248844601BC604700BF090E000001
:103CC00001B40248844601BC604700BFE512010010
:103CD00001B40248844601BC604700BFB70E000033
:103CE00001B40248844601BC604700BF891401004A
:103CF00001B40248844601BC604700BFED68010082
:103D000001B40248844601BC604700BF8937010006
:103D100001B40248844601BC604700BF6D0B01003E
:103D200001B40248844601BC604700BFDD0C0100BD
:103D300001B40248844601BC604700BF090E000080
:103D400001B40248844601BC604700BF53B900007B
:103D500001B40248844601BC604700BF69110100FC
:103D600001B40248844601BC604700BFCD0C01008D
:103D700001B40248844601BC604700BF894400008A
:103D800001B40248844601BC604700BFD9B00000BE
:103D900001B40248844601BC604700BFDD3F00001B
:103DA00001B40248844601BC604700BFC9A90000B5
:103DB00001B40248844601BC604700BFEDA5000085
:103DC00001B40248844601BC604700BF95730100FE
:103DD00001B40248844601BC604700BF75F800008A
:103DE00001B40248844601BC604700BFC1F700002F
:103DF00001B40248844601BC604700BFADAE00007C
:103E000001B40248844601BC604700BF21A90000FC
:103E100001B40248844601BC604700BF6DF6000053
:103E200001B40248844601BC604700BFDD0A0100BE
:103E300001B40248844601BC604700BFE90B0100A1
:103E400001B40248844601BC604700BFC16601005E
:103E500001B40248844601BC604700BFF935010047
:103E600001B40248844601BC604700BF61370100CD
:103E700001B40248844601BC604700BF4DF9000010
:103E800001B40248844601BC604700BF2D6C0100AC
:103E900001B40248844601BC604700BF9DA90000F0
:103EA00001B40248844601BC604700BF016C0100B8
:103EB00001B40248844601BC604700BFE927000006
:103EC00001B40248844601BC604700BF79970000F6
:103ED00001B40248844601BC604700BFE94C0100C0
:103EE00001B40248844601BC604700BF016701007D
:103EF00001B40248844601BC604700BF71B00000B5
:103F000001B40248844601BC604700BF01D70000ED
:103F100001B40248844601BC604700BFE9F60000D6
:103F200001B40248844601BC604700BF2144000040
:103F300001B40248844601BC604700BF85120100FD
:103F400001B40248844601BC604700BF8D82000076
:103F500001B40248844601BC604700BF79120100E9
:103F600001B40248844601BC604700BF496D0100AE
:103F700001B40248844601BC604700BF0934010017
:103F800001B40248844601BC604700BF053401000B
:103F900001B40248844601BC604700BF49B200003A
:103FA00001B40248844601BC604700BF51B800001C
:103FB00001B40248844601BC604700BF5976010045
:103FC00001B40248844601BC604700BFC56D0100D2
:103FD00001B40248844601BC604700BFBD0B01002C
:103FE00001B40248844601BC604700BFF90D0100DE
:103FF00001B40248844601BC604700BF3D71010026
:1040000001B40248844601BC604700BFB3520100BE
:1040100001B40248844601BC604700BFE9D40000F7
:1040200001B40248844601BC604700BFBD5C01008A
:1040300001B40248844601BC604700BFE917010093
:1040400001B40248844601BC604700BFCD4C01006A
:1040500001B40248844601BC604700BF116E0000F5
:1040600001B40248844601BC604700BFF535010039
:1040700001B40248844601BC604700BF75A9000036
:1040800001B40248844601BC604700BF01890000BA
:1040900001B40248844601BC604700BF8B52010056
:1040A00001B40248844601BC604700BFC1A50000BE
:1040B00001B40248844601BC604700BFC95C0100EE
:1040C00001B40248844601BC604700BFF9ED00001E
:1040D00001B40248844601BC604700BF0DB1001125
:1040E0000200000052B9001101000000C0B7001129
:1040F000020000004EB90011010000002041FF1F26
:1041000002000000C8B70011010000001062FF1F8C
:10411000020000004CB90011030000004461FF1FC1
:10412000120000000200000052B90011010000005E
:104130000CB80011020000004EB90011010000008F
:1041400009B800110200000016B8001103000000B9
:10415000D761FF1F020000004CB9001103000000EE
:10416000EC61FF1F020000004EB9001101000000C9
:1041700008B800110200000014B80011030000008C
:10418000AD61FF1F020000004CB9001103000000E8
:10419000CE61FF1F0200000052B9001101000000B3
:1041A0004CB80011020000004EB9001101000000DF
:1041B0006942FF1F020000005EB80011010000000C
:1041C00046B80011020000004EB9001101000000C5
:1041D0006842FF1F020000005CB8001101000000EF
:1041E000F461FF1F020000004EB900110100000041
:1041F0006742FF1F020000005AB8001101000000D2
:1042000036B80011020000004EB900110100000094
:104210006642FF1F0200000058B8001101000000B4
:1042200031B80011020000004EB900110100000079
:104230006542FF1F0200000056B800110100000097
:104240002CB80011020000004EB90011010000005E
:104250006442FF1F0200000054B80011010000007A
:1042600028B800110202020202020000D14A001125
:10427000954A00117CB8001190011D00180018002B
:10428000FFFF07010203040506020106000000000B
:10429000000000000000000000000000000000001E
:1042A000000000000000000003000000000100000A
:1042B00000000111FFFF00005048593600000000C7
:1042C000000000000B000500F0000000B400002812
:1042D000002800283075A000A000A000A000000861
:1042E0000008E001F00010001000100010001000A5
:1042F000100050005000500010001000D0070000C7
:10430000000000000F0001000500307507001000DC
:10431000010081FF00000000FF000000A56F0011F8
:10432000AD6D00113D6B0011FFFF0100FF000000AB
:10433000C19900113D970011559600110000000031
:104340000000000000000800040000003B0001081D
:104350005902E00188212800FF000000020000004F
:1043600052B900110100000018BA0011020000004B
:104370004EB9001101000000D943FF1F02000000E8
:104380004AB90011010000002C68FF1F0200000064
:104390004EB9001101000000D843FF1F02000000C9
:1043A00048B9001101000000D643FF1F02000000C1
:1043B0004EB9001101000000D443FF1F02000000AD
:1043C00046B9001101000000CC43FF1F180018007F
:1043D0001D00900102000003020200000200000024
:1043E00052B90011010000002CBA001102000000B7
:1043F0004EB90011010000001C44FF1F0200000024
:1044000044B900110000000000000000020000009C
:0E4410004CB90011030000004C68FF1F20FF94
:040000051FFF184180
:00000001FF
